:020000040800F2
:1030000000800020F1DD000823E700088DF30008B0
:1030100000000000000000000000000000000000B0
:1030200000000000000000000000000027E700088A
:10303000000000000000000025E7000885F30008FC
:1030400025DE000827DE000829DE00082BDE000848
:103050002DDE00082FDE000831DE000879F30008BD
:1030600035DE0008758B000839DE00083BDE0008FD
:103070003DDE00083FDE000841DE000843DE0008B8
:1030800045DE000847DE000849DE00084BDE000888
:103090004DDE0008858B000851DE000853DE000875
:1030A00055DE000857DE000859DE0008658B000871
:1030B0005DDE00085FDE000861DE000863DE0008F8
:1030C00001000000000000000A00000000000000F5
:1030D0006400000000000000E803000000000000A1
:1030E0001027000000000000A08601000000000082
:1030F00040420F0000000000809698000000000091
:1031000000E1F5050000000000CA9A3B0000000045
:1031100000E40B540200000000E8764817000000AD
:103120000010A5D4E800000000A0724E18090000AD
:1031300000407A10F35A00000080C6A47E8D030080
:103140000000C16FF286230000008A5D78456301AC
:10315000000064A7B3B6E00D0000E8890423C78A25
:0831600000487047F8FFFF1F53
:103168000348006803490A68101808607047C04699
:0831780080000020E40A0020A1
:1031800080B584B0039000F065F802900398019038
:103190000198401C002806D0FFE709480068019903
:1031A00008180190FFE7FFE700F054F80299401A71
:1031B0000199884201D2FFE7F6E704B080BDC0461E
:0431C000800000206B
:1031C40080B586B0059004A8002101701D480068F0
:1031D40000282FD0FFE71C4800681A4909687D229F
:1031E400D200039010460CF0ADFA03990290084601
:1031F40002990CF0A7FA0BF073FD002815D1FFE734
:10320400059803280CD8FFE705990020C2430190D4
:103214001046019A0AF007FF05980C49086003E07C
:1032240004A801210170FFE703E004A80121017053
:10323400FFE703E004A801210170FFE704A8007878
:1032440006B080BD8000002088000020840000209B
:0C325400014800687047C046E40A0020F2
:1032600080B582B001A8002101700B4801680122DD
:103270001302194301601046FFF7A4FF002804D091
:10328000FFE701A80121017002E005F0BBFBFFE7A9
:0C32900001A8007802B080BD00200240C0
:10329C0081B0009000988068012109070843034918
:1032AC0008400099886001B07047C046E8FFFF7F76
:1032BC0080B58CB00A9009A8002101700891079183
:1032CC0005910A98002804D1FFE70BA80121017091
:1032DC00B2E10A980069002809D0FFE70A98006952
:1032EC0001214905884201D1FFE7FFE7FFE70A9872
:1032FC00806D00280AD1FFE70A9804F017FE0A989F
:10330C000021C1650A9854228154FFE70A9800688D
:10331C000BF0F4FB002815D1FFE70A980068FFF7C3
:10332C00B7FFC7480068C7490CF008FA4000059081
:10333C00FFE70598002804D0FFE70598401E05908C
:10334C00F7E7FFE70A9800680BF0D8FB00280DD1CF
:10335C00FFE70A98816D1022114381650A98C16DAF
:10336C0001221143C16509A80270FFE70A980068A1
:10337C000AF0A1FD06900A98806DC006002800D5C1
:10338C004DE10698002800D049E10A98806D022191
:10339C0008430121090288430A9988650A98006844
:1033AC000BF0A4FB002835D1FFE70A980068C06831
:1033BC00182188430A998A6810430968C8600A98DA
:1033CC00006800690321890788430A9A53680B40F7
:1033DC00C018126810610A984068884219D0FFE73B
:1033EC000A98406801218907884212D0FFE70A98A1
:1033FC0040680121C90788420BD0FFE79248016859
:10340C000F22920491430A9B5B681340C918016018
:10341C00FFE7FFE70A98017E8903427ED20311433E
:10342C00827E52031143026B531E9A411203891878
:10343C00C2681143C07C00060028039107D5FFE742
:10344C000A9800690121C9078843029003E0012012
:10345C0040050290FFE70298039901430A982C2239
:10346C00805C400001430898084308900A9820218A
:10347C00405C012817D1FFE70A98807E002806D10E
:10348C00FFE7089801210904084308900AE00A980C
:10349C00816D2022114381650A98C16D012211436F
:1034AC00C165FFE7FFE70A98406A00280BD0FFE7E9
:1034BC000A98416A072292011140806A01430898D8
:1034CC0008430890FFE70A98016C426C1143826C28
:1034DC001143C06C01430798084307900A983C219C
:1034EC00405C012805D1FFE70798012108430790AC
:1034FC00FFE70A980068C0685449084008990843D7
:10350C000A990968C8600A9800680069504908401F
:10351C00079908430A99096808610A980168426B7F
:10352C0000200190084601990AF012FD0A980168E2
:10353C00826B48480090084600990AF009FD0A98E9
:10354C000069002808D1FFE70A980068816A0F22F9
:10355C00D243114381623CE00A980069012149057C
:10356C00884235D1FFE700200490FFE70498072834
:10357C0010D8FFE70A98006E04998900C8400F2103
:10358C0008400F2801D1FFE704E0FFE70498401C36
:10359C000490EBE70498012808D1FFE70A9800682B
:1035AC00816A0F22D2431143816210E00A980068AD
:1035BC00806A0A99CA699200121F1C231A400F23B1
:1035CC00DB4393400A6E134309688B62FFE7FFE706
:1035DC00FFE70A980068C0681F49084008998842AC
:1035EC000CD1FFE70A980021C1650A98806D012172
:1035FC000843022188430A9988650FE00A98806D78
:10360C0010210843022188430A9988650A98C16DE4
:10361C0001221143C16509A80270FFE708E00A986E
:10362C00816D10221143816509A801210170FFE70A
:10363C0009980BA90870FFE70BA800780CB080BDA7
:10364C0088000020400D0300082701401902FEFFEE
:0C365C0002FCFFDF04FFFF07E7FF3F83D5
:1036680080B586B0049003910292049800680AF02D
:1036780024FC00286FD1FFE7FFE704985421405C41
:10368800012804D1FFE705A8022101706BE0049826
:10369800542101224254FFE7FFE704980068C068FC
:1036A800C007002813D1FFE7049800680BF020FA40
:1036B800002805D0FFE70498006800F0CFF8FFE77E
:1036C80004980068C16801221143C160FFE70498AB
:1036D80000F056F801A90870087800283AD1FFE7E9
:1036E8000498806D01210902084321490840049982
:1036F800886504980021C1650498006D1D49C16260
:103708000498006D1C4901630498006D1B494163CE
:10371800049800681C210160FFE7049854210022E6
:103728004254FFE704980068416810221143416041
:103738000498016D00684030039A029B0090084687
:1037480000990AF07DFC01A908700498006800F04F
:1037580077F8FFE703E001A802210170FFE701986D
:1037680005A90870FFE705A8007806B080BDC04627
:10377800FEF1FFFFE1EB000883DF000899DF000896
:1037880080B584B00290029800680BF0B1F9002867
:103798004BD1FFE7029800688068284908420DD09D
:1037A800FFE70298816D1022114381650298C16D6F
:1037B80001221143C16503A802703AE0029800682B
:1037C80000F06EF80298407E01282DD0FFE7FFF741
:1037D8003DFD0190FFE7029800680068C0070028D7
:1037E80021D1FFE7029800680BF082F9002805D183
:1037F800FFE70298006800F053F8FFE7FFF726FD9F
:103808000199401A03280DD3FFE70298816D102211
:10381800114381650298C16D01221143C16503A856
:10382800027006E0D7E7FFE7FFE703A80021017071
:10383800FFE703A8007804B080BDC04617000080E9
:1038480081B000900098806803490840001D0099E5
:0C385800886001B07047C046E8FFFF7FA9
:1038640081B000900098806803490840801C00994A
:0C387400886001B07047C046E8FFFF7F8D
:1038800083B0029001910092029840690199090267
:103890008843009A0A4003490A401043029948614C
:0838A00003B0704700FFFF07B1
:1038A80081B000900098806803490840401C009946
:0C38B800886001B07047C046E8FFFF7F49
:1038C40082B00190009100980349084001998A6AE6
:0C38D40002438A6202B07047FFFF070049
:1038E00082B0019000910098C043044908430199B7
:1038F0008A6A02408A6202B07047C0460000F8FF40
:1039000080B5A4B02290219120A8002101701E91C1
:10391000229800690121C907884206D0FFE7229852
:103920000069FB49884201D1FFE700E0FFE7FFE7BC
:1039300022985421405C012804D1FFE723A80221EA
:1039400001701CE22298542101224254FFE7FFE754
:10395000229800680AF0B5FA002800D0FCE121980E
:103960004068022800D19EE1229800690121C90720
:10397000884206D0FFE722980069E549884207D1CE
:10398000FFE72298006821990968FFF79BFF1DE176
:103990002298006E21994A681F231A400F239340F2
:1039A00098430968490300291D9008D1FFE7219831
:1039B00000681F2189060840800E1C90E7E02198CE
:1039C0000078C007002803D0FFE700201B90DBE051
:1039D000219800788007002803D5FFE701201A907E
:1039E000CFE0219800784007002803D5FFE70220A8
:1039F0001990C3E0219800780007002803D5FFE75D
:103A000003201890B7E021980078C006002803D55D
:103A1000FFE704201790ABE021980078800600288B
:103A200003D5FFE7052016909FE021980078400617
:103A3000002803D5FFE70620159093E02198007831
:103A40000006002803D5FFE70720149087E021989F
:103A50004078C007002803D0FFE7082013907BE0E0
:103A6000219840788007002803D5FFE709201290AD
:103A70006FE0219840784007002803D5FFE70A202F
:103A8000119063E0219840780007002803D5FFE7F4
:103A90000B20109057E021984078C006002803D5ED
:103AA000FFE70C200F904BE021984078800600281B
:103AB00003D5FFE70D200E903FE0219840784006A7
:103AC000002803D5FFE70E200D9033E021984078C1
:103AD0000006002803D5FFE70F200C9027E021986F
:103AE0008078C007002803D0FFE710200B901BE070
:103AF000219880788007002803D5FFE711200A90DD
:103B00000FE0219800680121890408401222002357
:103B100088420993089201D00998089008980A9061
:103B2000FFE70A980B90FFE70B980C90FFE70C98C3
:103B30000D90FFE70D980E90FFE70E980F90FFE7AE
:103B40000F981090FFE710981190FFE711981290CE
:103B5000FFE712981390FFE713981490FFE714986B
:103B60001590FFE715981690FFE716981790FFE756
:103B700017981890FFE718981990FFE719981A906E
:103B8000FFE71A981B90FFE71B981C90FFE71C9813
:103B9000219949681F22114088401D9901432298AC
:103BA0000166219840688008401C2299C9698842B2
:103BB0000BD8FFE72298006821994A6809680791A5
:103BC0001146079A0AF01AFAFFE7FFE72298006801
:103BD00021990A68896806911146069AFFF750FEF6
:103BE0002198C078000600285CD5FFE767480AF0F6
:103BF000FCF91F90219800686549884220D1FFE7B1
:103C00001FA88078000600281AD4FFE71F9801211A
:103C1000C90508435D490590084605990BF042F82F
:103C20005E4800685E490BF08FFD1E90FFE71E980E
:103C3000002804D0FFE71E98401E1E90F7E730E0F2
:103C4000219800685349884211D1FFE71FA8C07826
:103C5000C00700280BD1FFE71F9801210906084380
:103C60004A490490084604990BF01CF818E0219882
:103C700000684949884211D1FFE71FA880784006B3
:103C800000280BD4FFE71F980121890508433F490D
:103C90000390084603990BF005F800E0FFE7FFE703
:103CA000FFE7FFE757E0229800690121C907884232
:103CB00006D0FFE7229800693349884207D1FFE721
:103CC0002298006821990968FFF70AFEFFE721980A
:103CD000C078000600283DD5FFE72C480AF085F99A
:103CE0001F90219800682A4988420BD1FFE71F984E
:103CF0000121C905884325490290084602990AF026
:103D0000D1FF26E021980068224988420DD101E0C8
:103D1000040000801F980121090688431B49019077
:103D2000084601990AF0BEFF12E0219800681A497E
:103D300088420BD1FFE71F98012189058843134969
:103D40000090084600990AF0ADFF00E0FFE7FFE7AA
:103D5000FFE7FFE7FFE708E02298816D202211438B
:103D6000816520A801210170FFE7FFE72298542117
:103D700000224254FFE7209823A90870FFE723A8F8
:103D8000007824B080BDC0460400008008270140B0
:103D9000001000B0004000B8002000B488000020EF
:043DA000400D0300CF
:103DA40080B586B0049000200290FFE70498542167
:103DB400405C012804D1FFE705A8022101706DE0F1
:103DC4000498542101224254FFE7FFE704980AF0C3
:103DD400ABFE03A90870049800680AF079FF002874
:103DE4004CD1FFE70498806D0221084301210A02A7
:103DF4009043049A906504980068C06803221040B8
:103E0400019004980068C3689343C36004980068F1
:103E14008268C9070A438260FFE7049800680AF0D1
:103E24004DFF00281BD0FFE70298401C0290029827
:103E34001C49884212D3FFE70498806D102108437F
:103E44000221884304998865FFE7049854210022DD
:103E54004254FFE705A8012101701FE0DDE7019846
:103E640004990968CA680243CA600498806D0121F4
:103E74000843022188430499886505E00498816D0C
:103E8400102211438165FFE7FFE7049854210022C3
:103E94004254FFE7039805A90870FFE705A80078D6
:083EA40006B080BD00F202002F
:103EAC0081B001466A46107010781F221040012222
:103EBC0082400248026001B07047C04680E100E0D9
:103ECC0070B582B0024601AB18700091187840B200
:103EDC0000281BD5FFE701A801780F2211400839F3
:103EEC000323DB431940174C0959007840B285076E
:103EFC00ED0EFF26AE40B143009EB601F6B2AE40C9
:103F0C003143104008381840015116E001A80178DF
:103F1C0049B20322D2431140094BC958007840B230
:103F2C008407E40EFF25A540A943009DAD01EDB229
:103F3C00A54029431040C150FFE702B070BDC046F8
:083F4C0000E400E01CED00E0C0
:103F540081B001466A46107010781F221040012279
:103F640082400248026001B07047C04600E100E0B0
:103F740080B584B002900298401E000E002803D041
:103F8400FFE70120039013E00298401E0A490860ED
:103F94000020C1430322019008461146FFF794FF15
:103FA4000648019901600648072202600391FFE771
:103FB400039804B080BDC04614E000E018E000E0BF
:043FC40010E000E029
:103FC80080B584B003905848006802900398006850
:103FD8000068019002980399096C1C221140C8409E
:103FE8004007002828D5FFE701A8007840070028E7
:103FF80022D5FFE70398006800688006002807D4E8
:10400800FFE7039800680168042291430160FFE715
:104018000398006C1C210840042181404348026831
:104028000A4302600398006B002804D0FFE7039856
:10403800016B8847FFE774E002980399096C1C221A
:104048001140C8408007002832D5FFE701A8007852
:10405800800700282CD5FFE70398006800688006D1
:1040680000280BD4FFE70398006801680A229143EF
:1040780001600398252101224254FFE70398006C50
:104088001C21084002218140284802680A43026036
:10409800FFE70398242100224254FFE70398C06AEF
:1040A800002804D0FFE70398C16A8847FFE737E094
:1040B80002980399096C1C221140C8400007002887
:1040C8002CD5FFE701A800780007002826D5FFE7D0
:1040D8000398006801680E22914301600398006C00
:1040E8001C21084001210A468240104803681343F6
:1040F80003600398C163039825228154FFE703985E
:10410800242100224254FFE70398406B002804D082
:10411800FFE70398416B8847FFE700E0FFE7FFE709
:10412800FFE704B080BDC046000002400400024022
:1041380084B003900291019200930398C16C806C43
:1041480041600398006D002805D0FFE70398816D52
:10415800406D4160FFE70398006C1C210840012175
:104168008140104802680A43026000980399096870
:10417800486003988068102809D1FFE701980399DF
:1041880009688860029803990968C86008E002987D
:10419800039909688860019803990968C860FFE76E
:0841A80004B07047040002405E
:1041B00080B584B002900298002804D1FFE703A8DC
:1041C000012101706DE002980168384A89181422B3
:1041D0000190084611460BF0B7FA80000199086477
:1041E0000298252202238354029800680268304B0B
:1041F0001A40026002988268C3681A4303691A432E
:1042000043691A4383691A43C3691A43036A1A4309
:104210000068036813430360029800F04BF80298AB
:10422000806801218903884204D1FFE702980021B8
:104230004160FFE702980179406C01600298C16C0F
:10424000806C416002984068002811D0FFE7029816
:10425000406804280CD8FFE7029800F04DF8029857
:10426000006D002101600298816D406D416007E0A2
:104270000298002101650298416502988165FFE777
:1042800002980021C1630298252101224254FFE7D0
:104290000298242100224254FFE703A80021017064
:1042A000FFE703A8007804B080BDC046F8FFFDBF5B
:0442B0000F80FFFF7D
:1042B40080B582B0019001980078083814210BF081
:1042C40041FA00900198016C03229143074A89182E
:1042D400416401980649816400981C210840012129
:1042E40081400198C16402B080BDC046000802400C
:0442F40080080240FC
:1042F80082B00190019800790090009880000849E8
:104308004018019908650198064941650098401EC2
:1043180003210840012181400198816502B070475E
:08432800FC08024040090240BC
:1043300010B584B0194614460390019300920748C3
:10434000026801231A4302600098039A1060BFF3C9
:104350006F8F0198039A506004B010BD1420024082
:1043600080B584B00290FEF775FF02994018009066
:10437000FFE736480068012109040840000C0028C6
:104380000BD0FFE7FEF766FF0099884204D3FFE7F2
:1043900003A80321017054E0EBE72C4800682C4986
:1043A000084001902B4800680121890708400199C5
:1043B00001430191FFE701A8C0780006800F0028A3
:1043C00009D0FFE7019803218907084021490A68BD
:1043D00002430A60FFE701988000002807D0FFE74A
:1043E000019803218907884318490860FFE7FFE720
:1043F0000198002807D0FFE701981749486003A8F3
:10440000012101701DE0FEF725FF02994018009080
:10441000FFE70E480068012189040840800C00284D
:104420000BD0FFE7FEF716FF0099884204D3FFE7A1
:1044300003A80321017004E0EBE703A80021017049
:10444000FFE703A8007804B080BDC04610200240FA
:0C445000FA83000018200240900D0020AC
:10445C00B0B588B01C4615460690059103930292A0
:10446C00FFE720480078012804D1FFE707A80221C4
:10447C00017033E01B4801210170FFE7FFE7194889
:10448C00002141601848FFF765FF01A90870087802
:10449C0000281AD1FFE70698012806D1FFE70598F6
:1044AC00039B029AFFF73EFF04E00598029900F087
:1044BC001FF8FFE70C48FFF74DFF01A9087006989D
:1044CC000A490A6882430A60FFE7FFE705480021B2
:1044DC000170FFE7019807A90870FFE707A80078AB
:1044EC0008B0B0BD900D00208813000014200240CD
:1044FC0008B4024B9C4608BC6047C046050000202F
:10450C0081B06846012101700C4800684000002809
:10451C0010D5FFE70A480B4901600B4901600748B9
:10452C0000684000002804D4FFE7684600210170B1
:10453C00FFE7FFE76846007801B07047142002409F
:0C454C000C2002403B2A19087F6E5D4CD9
:1045580081B06846002101700C480068C00F00282F
:1045680010D0FFE70A480B4901600B490160074872
:104578000068C00F002804D0FFE7684601210170D9
:10458800FFE7FFE76846007801B070471420024053
:0C4598000820024023016745AB89EFCDED
:1045A40081B06846012101700848026889070A43FE
:1045B400026000684000002804D5FFE76846002137
:1045C4000170FFE76846007801B07047142002408C
:1045D40081B068460121017008480268C9070A438E
:1045E40002600068C00F002804D0FFE7684600217D
:1045F4000170FFE76846007801B07047142002405C
:1046040082B00A480068C0B200900098AA2807D077
:10461400FFE70098CC2803D0FFE7BB20019002E01D
:1046240000980190FFE7019802B0704720200240F3
:1046340002480168024A1143016070471420024095
:04464400040001006D
:104648008AB00990089100200790FFE70898006851
:104658000799C840002800D148E1089800680799E0
:1046680001228A40104006900698002800D139E1BE
:1046780008984068022805D0FFE708984068122883
:1046880020D1FFE709980799C90889004018006AEE
:10469800059007984007C00E0F2181400598884370
:1046A80005900898006907994907C90E8840059937
:1046B8000143059105980999079AD208920089182B
:1046C8000862FFE7099800680590079840000321F1
:1046D8000A4682400598904305900898406808402B
:1046E800079949008840059901430591059809995A
:1046F80008600898406801280FD0FFE708984068CC
:1047080002280AD0FFE708984068112805D0FFE77B
:104718000898406812282CD1FFE70998806805900E
:104728000798400003218140059888430590089820
:10473800C068079949008840059901430591059883
:104748000999886009984068059007980121814077
:10475800059888430590089840681021084000098A
:10476800079988400599014305910598099948607A
:10477800FFE70998C0680590079840000321814029
:1047880005988843059008988068079949008840EB
:1047980005990143059105980999C8600898C07959
:1047A800C006002800D49CE007980321884350499C
:1047B8004058059007988007C00E0F218140059842
:1047C80088430590099805210907884203D1FFE726
:1047D8000020049022E009984649884203D1FFE767
:1047E8000120039017E009984349884203D1FFE765
:1047F800022002900CE009984049032205238842D0
:104808000193009201D00198009000980290FFE770
:1048180002980390FFE703980490FFE7049807992C
:104828008907C90E8840059901430591059807999C
:10483800032291432E4A8850314800680590069813
:1048480005998143059108988079C007002805D00B
:10485800FFE70698059901430591FFE70598284960
:1048680008602848006805900698059981430591D5
:10487800089880798007002805D5FFE706980599EC
:1048880001430591FFE705981E4908601E48006826
:104898000590069805998143059108988079C00686
:1048A800002805D5FFE70698059901430591FFE71C
:1048B80005981549086015480068059006980599F7
:1048C80081430591089880798006002805D5FFE77F
:1048D8000698059901430591FFE705980B4908607B
:1048E800FFE7FFE70798401C0790AFE60AB070475C
:1048F800601802400004005000080050000C0050EE
:10490800801802408418024000180240041802402F
:1049180080B582B0014601AA10800F48006812884D
:10492800104208D0FFE701A801880B4A11600088EF
:104938000AF0F4F9FFE70948006801A90988084264
:1049480008D0FFE701A80188044A116000880AF02E
:10495800FFFCFFE702B080BD0C18024010180240AF
:1049680080B582B0019001980721016001984168E3
:10497800024608320C30009008461146009A00F0B2
:104988000FF8FFF73BFE0199086100F077F90199EC
:10499800886101980149416102B080BD00604F07FC
:1049A80083B0029001910092029801280DD1FFE78F
:1049B8000E4801683F221140019B196000681104EC
:1049C8000840000C009908600CE0074801683F2285
:1049D8001140019B1960006811040840000C0099FF
:1049E8000860FFE703B07047302002402C200240E7
:1049F80080B586B004900391FFE73048007801281D
:104A080004D1FFE705A80221017052E02B480121DB
:104A18000170FFE7FFE72948002141602848FFF7B8
:104A28009BFC02A908700878002839D1FFE7049890
:104A38000068042808D1FFE7FFF7F8FD2048FFF7D2
:104A48008BFC02A908702AE003980021C943016081
:104A5800049840680190FFE7019804994A688968BA
:104A68005118884215D2FFE7019800F02DF8144834
:104A7800FFF772FC02A908700878002804D0FFE745
:104A880001980399086004E0FFE70198401C019031
:104A9800E2E70C480168022291430160FFE7FFE763
:104AA800FFE7064800210170FFE7029805A9087092
:104AB800FFE705A8007806B080BDC046900D00202D
:084AC8008813000014200240D5
:104AD00082B00190074801683F22D20091430091C3
:104AE0000099019AD2000A4303490A43026002B0C6
:0C4AF0007047C046142002400200010084
:104AFC0080B58AB00890FFE742480078012804D1BD
:104B0C00FFE709A80221017077E03E4801210170FE
:104B1C00FFE7FFE73B480021416008980078C00799
:104B2C0000280BD0FFE7089841688268C0680590A0
:104B3C0008461146059A00F06BF8FFE708980068E4
:104B4C000621084006280BD1FFE7089841698269C5
:104B5C000069049008461146049A00F075F826E0A6
:104B6C0008980078800700280BD5FFE700F084F840
:104B7C000790079808990A690390039900F064F864
:104B8C0014E008980078400700280DD5FFE7FFF7E0
:104B9C0033FD0790089841698069079A029008468E
:104BAC00029900F051F800E0FFE7FFE7FFE7164835
:104BBC00FFF7D0FB06A908700878002814D1FFE78E
:104BCC001248016801225204114301600E49019000
:104BDC0008460092FFF7BEFB06A908700198016811
:104BEC00009A91430160FFE7FFE70648002101703E
:104BFC00FFE7069809A90870FFE709A800780AB032
:104C0C0080BDC046900D0020881300001420024087
:104C1C0083B00290019100920298012807D0FFE71F
:104C2C0000980004019908430649086006E00098C2
:104C3C0000040199084302490860FFE703B070477C
:084C4C002C2002403020024040
:104C540084B003900291019208480168009103997D
:104C6400009A8A43FF218A4300920099029A1143D1
:104C7400019A1143016004B07047C04620200240ED
:104C840081B004480068044908400090009801B0CD
:0C4C94007047C0462020024000604F071F
:104CA0000348016801221202914301607047C04627
:044CB0000070004050
:104CB4000348016801221202114301607047C04693
:044CC400007000403C
:104CC800024800680721090308407047081002409D
:104CD80010B588B006900698002804D1FFE707A809
:104CE800012101702EE306980078C007002800D142
:104CF80088E0FC480068382108400490FA480068B9
:104D08000321084003900498102804D1FFE7039872
:104D1800032804D0FFE70498082810D1FFE7F848D3
:104D280000688003002809D5FFE706984068002836
:104D380004D1FFE707A80121017003E361E0FFE761
:104D48000698406801210904884207D1FFE7EC482A
:104D5800016801221204114301601DE006984068B1
:104D68000521090488420BD1FFE7E54801680122C3
:104D780093041943016001681204114301600AE0B9
:104D8800DF48016801221304994301600168920415
:104D980091430160FFE7FFE7FFE7069840680028B6
:104DA80017D0FFE7FEF752FA0590FFE7D4480068EE
:104DB800800300280CD4FFE7FEF748FA0599401A4B
:104DC800652804D3FFE707A803210170BAE2EDE7DD
:104DD80016E0FEF73BFA0590FFE7C9480068800334
:104DE80000280CD5FFE7FEF731FA0599401A652827
:104DF80004D3FFE707A803210170A3E2EDE7FFE76B
:104E0800FFE7FFE7069800788007002800D4A3E0B2
:104E1800B4480068382108400490B348006803216A
:104E2800084003900498102804D1FFE7039802284B
:104E380004D0FFE7049800283BD1FFE7B04800689A
:104E48004005002809D5FFE70698C068002804D166
:104E5800FFE707A80121017074E2AA4801687F22D0
:104E680012029143069A5269120211430160049892
:104E7800002811D1FFE7A24801680722D202914316
:104E8800069B1B691943016000681040C00A9E49CF
:104E9800C1409E480160FFE79D480068FEF78EF913
:104EA800002804D0FFE707A8012101704AE2FFE7C4
:104EB80051E00698C06800282FD0FFE790480168A5
:104EC8000722D2029143069A1269114301600168D0
:104ED8000122120211430160FEF7B8F90590FFE7BD
:104EE80087480068400500280CD4FFE7FEF7AEF9B4
:104EF8000599401A032804D3FFE707A80321017086
:104F080020E2EDE77F4801687F2212029143069A6A
:104F180052691202114301601CE0794801680122BC
:104F2800120291430160FEF791F90590FFE774487A
:104F38000068400500280CD5FFE7FEF787F90599BA
:104F4800401A032804D3FFE707A803210170F9E1F9
:104F5800EDE7FFE7FFE7FFE706980078000700287E
:104F680056D5FFE7F948006838210840182810D1BD
:104F7800FFE7F94800688007002809D5FFE7069889
:104F88008069002804D1FFE707A801210170D9E151
:104F98003DE00698806900281CD0FFE7EE480168CC
:104FA800012211430160FEF751F90590FFE7EA4835
:104FB8000068800700280CD4FFE7FEF747F9059939
:104FC800401A032804D3FFE707A803210170B9E1B9
:104FD800EDE71BE0E0480168012291430160FEF71C
:104FE80035F90590FFE7DC480068800700280CD5F4
:104FF800FFE7FEF72BF90599401A032804D3FFE7CA
:1050080007A8032101709DE1EDE7FFE7FFE7FFE750
:10501800069800784007002800D4CAE002A80021BA
:105028000170CA48006838210840202810D1FFE7DD
:10503800CC4800688007002809D5FFE706988068F3
:10504800002804D1FFE707A8012101707AE1AFE049
:10505800C2480068C000002810D4FFE7FFE7BF4837
:105068000168012212071143016000681040019095
:105078000198FFE702A801210170FFE7B84800681E
:10508800C00500281DD4FFE7B548016801221202B7
:1050980011430160FEF7DAF80590FFE7B0480068B1
:1050A800C00500280CD4FFE7FEF7D0F80599401A90
:1050B800032804D3FFE707A80321017042E1EDE7C5
:1050C800FFE7FFE706988068012806D1FFE7A548B3
:1050D800016801221143016027E0069880680528CD
:1050E80018D103E0081002400C1002409D480168E6
:1050F800042211430160016801221143016013E099
:1051080000100240041002400024F400880000202F
:1051180084000020934801680122914301600168DE
:10512800042291430160FFE7FFE7FFE706988068E4
:10513800002818D0FFE7FEF789F80590FFE78948AF
:105148000068800700280DD4FFE7FEF77FF805996F
:10515800401A8549884204D3FFE707A80321017054
:10516800F0E0ECE717E0FEF771F80590FFE77D48FF
:105178000068800700280DD5FFE7FEF767F8059956
:10518800401A7949884204D3FFE707A80321017030
:10519800D8E0ECE7FFE702A80078012807D1FFE78D
:1051A8006E4801680122120791430160FFE7FFE79B
:1051B800FFE70698C069002800D1BFE0634800688F
:1051C8003821084010287AD0FFE70698C0690228DD
:1051D8004ED1FFE75F480168012212069143016042
:1051E800FEF734F80590FFE75A4800688001002868
:1051F8000CD5FFE7FEF72AF80599401A032804D3CF
:10520800FFE707A8032101709CE0EDE7504801681B
:10521800574A1140069A136A546A2343946A24022F
:105228002343D46A2343126B13431943016049494A
:105238000A6801231C0622430A6001681A07114301
:105248000160FEF703F80590FFE742480068800117
:1052580000280CD4FFE7FDF7F9FF0599401A032849
:1052680004D3FFE707A8032101706BE0EDE725E011
:1052780038480168012212069143016034480168E8
:105288000322914301600168384A11400160FDF72B
:10529800DDFF0590FFE72F480068800100280CD546
:1052A800FFE7FDF7D3FF0599401A032804D3FFE76A
:1052B80007A80321017045E0EDE7FFE73DE0069808
:1052C800C069012804D1FFE707A80121017039E06E
:1052D8001F48006803900398032108400699096A4B
:1052E800884224D1FFE70398702108400699496A4B
:1052F80088421CD1FFE703987F21090208400699DC
:10530800896A0902884212D1FFE703981F214904DC
:1053180008400699C96A884209D1FFE7039807211E
:10532800490708400699096B884204D0FFE707A897
:105338000121017006E0FFE7FFE7FFE707A800216A
:105348000170FFE707A8007808B010BD08100240F8
:105358000C10024000100240601002403C10024055
:10536800007000405C10024089130000FFFFFEEF50
:045378008C80C11F45
:10537C0080B588B0404800688006400F00280FD1E7
:10538C00FFE7414800680721C9020840C00A012113
:10539C008140039103993B480AF0D0F9029067E0F1
:1053AC003548006838210840082803D1FFE7344805
:1053BC0002905CE0304800683821084010283AD14F
:1053CC00FFE72E4801680322114006910068702106
:1053DC0008400009401C049006980228019011D046
:1053EC00FFE7019803280ED1FFE7049924480AF03F
:1053FC00A5F9224909687F2212021140090A41438A
:10540C0007910DE0FFE704991E480AF097F91B4934
:10541C0009687F2212021140090A41430791FFE7F4
:10542C0016480068400F401C0590079805990AF033
:10543C0085F902901AE010480068382108402028AD
:10544C0004D1FFE70120C00302900EE00A48006877
:10545C0038210840182804D1FFE77D200002029073
:10546C0002E000200290FFE7FFE7FFE7FFE7FFE71E
:10547C00029808B080BDC046081002400C100240D3
:0C548C0000127A000024F400001002401E
:1054980080B584B0029001910298002804D1FFE7FA
:1054A80003A8012101700CE10198884909680722C5
:1054B8001140884221D9FFE78448016807229143B7
:1054C800019A11430160FDF7C1FE0090FFE77F4894
:1054D800006807210840019988420DD0FFE7FDF7D1
:1054E800B5FE0099401A8149884204D3FFE703A812
:1054F80003210170E5E0EAE7FFE7029800788007FA
:10550800002817D5FFE7029800784007002807D53C
:10551800FFE76F4801680722120311430160FFE7A4
:105528006B4801680F2212029143029A9268114354
:105538000160FFE702980078C007002872D0FFE7F3
:105548000298406801280BD1FFE76448006880038F
:10555800002804D4FFE703A801210170B1E03DE071
:105568000298406802280BD1FFE75C480068800178
:10557800002804D4FFE703A801210170A1E02CE072
:105588000298406800280BD1FFE75448006840059E
:10559800002804D4FFE703A80121017091E01BE073
:1055A8000298406803280BD1FFE74B480068800742
:1055B800002804D4FFE703A80121017081E00AE074
:1055C800444800688007002804D4FFE703A80121A5
:1055D800017076E0FFE7FFE7FFE7FFE73C48016877
:1055E80007229143029A526811430160FDF72EFE8B
:1055F8000090FFE73648006838210840029949685A
:10560800C90088420DD0FFE7FDF720FE0099401A37
:105618003649884204D3FFE703A80321017050E00C
:10562800E8E7FFE7019829490968072211408842FD
:1056380021D2FFE72548016807229143019A1143C7
:105648000160FDF703FE0090FFE72048006807218E
:105658000840019988420DD0FFE7FDF7F7FD009952
:10566800401A2249884204D3FFE703A803210170A6
:1056780027E0EAE7FFE702980078400700280AD504
:10568800FFE713480168072212039143029AD26880
:1056980011430160FFE7FFF76DFE0D4909680F220E
:1056A8001202114089090E4A51581F221140C84060
:1056B8000C4908600C480068FDF780FD03A90870D4
:1056C800FFE703A8007804B080BDC0460020024070
:1056D800081002405C1002406010024000100240B6
:1056E8009CD900088800002084000020891300004D
:0C56F800014800687047C0468800002090
:1057040080B584B002901B48016803225202914381
:10571400029A11430160029801214902884221D171
:10572400FFE71548006806214143144800900846E5
:1057340000990AF007F8401C0190FFE71048006840
:10574400400500280DD5FFE70198002804D0FFE7A5
:105754000198401E019003E003A80321017005E0B5
:10576400ECE7FFE703A800210170FFE703A8007836
:1057740004B080BD007000408800002040420F004B
:04578400147000405D
:1057880080B582B0FFF7B4FF0190FFF799FA000BDC
:105798008000044908581F2108400199C140084663
:0857A80002B080BDDCD900084D
:1057B00080B584B0039001A80021017003980068AF
:1057C000C0684006002830D4FFE703980068C1682D
:1057D00080221143C160FDF73DFD0290FFE7039871
:1057E0000068C068002140060028009107D4FFE748
:1057F00001A80078C01E411E88410090FFE7009874
:10580000C007002810D0FFE7FDF724FD0299401AD9
:105810000849884207D3FFE701A8032101700398D4
:1058200029228154FFE7DAE7FFE701A8007804B0F6
:0858300080BDC046E903000041
:1058380080B582B001906846002101701A4801685D
:1058480080229143016019480068800600280ED420
:10585800FFE7019800F01AFB002807D0FFE701983E
:1058680029210322425468460270FFE717E00F48D7
:105878000168202291430160019800F007FB00288D
:1058880007D0FFE701982921032242546846027095
:10589800FFE706480168202211430160FFE76846D8
:1058A800007802B080BDC0460C280040182800408F
:1058B80080B588B0079004A80021017003A8017082
:1058C800079880788007002800D49DE002A800216E
:1058D800017084480068C000002810D4FFE7FFE783
:1058E80080480168012212071143016000681040D6
:1058F80001900198FFE702A801210170FFE77A48AB
:1059080001680122120211430160FDF79FFC059016
:10591800FFE775480068C00500280CD4FFE7FDF7CD
:1059280095FC0599401A032804D3FFE704A803212E
:10593800017000E0EDE704A80078002853D1FFE7E4
:105948006A48006803210902084006900698002862
:1059580017D0FFE7069807998969884211D0FFE7B1
:1059680062480168032212029143069101680122EC
:1059780012041143016001689143016006990160B6
:10598800FFE706A80078C007002818D0FFE7FDF752
:105998005DFC0590FFE755480068800700280DD496
:1059A800FFE7FDF753FC0599401A5149884204D393
:1059B800FFE704A80321017000E0ECE7FFE704A873
:1059C800007800280AD1FFE748480168032212023C
:1059D8009143079A92691143016003E0049803A96F
:1059E8000870FFE703E0049803A90870FFE702A81E
:1059F8000078012807D1FFE73A4801680122120719
:105A080091430160FFE7FFE707980078C007002887
:105A180009D0FFE73748016803229143079A526883
:105A280011430160FFE7079800788007002809D52F
:105A3800FFE7304801680C229143079A92681143A6
:105A48000160FFE707980078400600280AD5FFE7BD
:105A580028480168032212039143079AD268114328
:105A68000160FFE7079840784006002818D5FFE74F
:105A780020480168032292079143079A526911430B
:105A880001600798406901218907884207D1FFE72B
:105A9800194801680122120411430160FFE7FFE77A
:105AA800079840780007002818D5FFE711480168D3
:105AB800032292039143079A1269114301600798E0
:105AC800006901218903884207D1FFE70A48016874
:105AD8000122120411430160FFE7FFE703A80078E1
:105AE80008B080BD3C100240007000405C100240CD
:0C5AF80089130000541002400C10024002
:105B040080B582B001906846012101700198002897
:105B140071D0FFE701982921405C00280CD1FFE7F0
:105B2400019828210022425401981121C9024160A0
:105B3400019802F01BFFFFE7019829210222425439
:105B4400FFE701980068CA21416201980068532167
:105B54004162FFE70198FFF729FE6946087008785B
:105B6400002837D1FFE7019800688169244A114071
:105B740081610198816842691143C26911430068D7
:105B840082690A4382610198016900680161019890
:105B9400C1680904006802690A4302610198FFF7B9
:105BA40049FE694608700878002812D1FFE7019879
:105BB4000068816907225207914381610198416A13
:105BC400026A114382691143006882690A4382614F
:105BD400FFE7FFE7FFE701980068FF214162FFE765
:105BE40068460078002805D1FFE7019829210122A1
:105BF4004254FFE7FFE76846007802B080BDC04624
:045C0400BFFF8FFB54
:105C080080B588B0069005910492FFE70698282190
:105C1800405C012804D1FFE707A80221017097E042
:105C28000698282101224254FFE7FFE70698292118
:105C380002224254FFE706980068CA21416206988A
:105C4800006853214162FFE70698FFF7ADFD02A9FE
:105C580008700878002861D1FFE70498002828D147
:105C6800FFE70698006880694006002801D5FFE72D
:105C780003E005980021C170FFE70598007808F057
:105C8800ADFA0004059949780190084608F0A6FA8B
:105C9800000201990818059989780090084608F0CB
:105CA8009DFA009908180599C97889050843039051
:105CB80018E00698006880694006002801D5FFE7CB
:105CC80003E005980021C170FFE7059801780904F1
:105CD80042781202891882788918C07880050143B1
:105CE8000391FFE703981C49084006990968086072
:105CF80006980068816901229204914381610598A0
:105D0800C168006901430698006882690A43826194
:105D18000698FFF78DFD02A90870FFE7FFE70698D0
:105D28000068FF214162FFE702A80078002805D13A
:105D3800FFE70698292101224254FFE7FFE706986A
:105D4800282100224254FFE7029807A90870FFE7BC
:0C5D580007A8007808B080BD7F7F7F00A6
:105D640080B588B0069005910492FFE70698282133
:105D7400405C012804D1FFE707A80221017080E0FC
:105D84000698282101224254FFE7FFE706982921BB
:105D940002224254049800280DD1FFE70598407868
:105DA400C006002807D5FFE705984178EF22114087
:105DB4000A314170FFE7049800281CD1FFE70598D9
:105DC400C07808F00DFA0004059949780190084656
:105DD40008F006FA000201990818059989780090DC
:105DE400084608F0FDF9009908180599097849034F
:105DF400084303900CE00598C17809044278120224
:105E04008918827889180078400301430391FFE7D9
:105E1400FFE706980068CA2141620698006853218A
:105E24004162FFE70698FFF7C1FC02A908700878F1
:105E340000280CD1FFE70398144908400699096823
:105E440048600698FFF7F6FC02A90870FFE7FFE731
:105E540006980068FF214162FFE702A80078002845
:105E640005D1FFE70698292101224254FFE7FFE705
:105E74000698282100224254FFE7029807A90870D7
:105E8400FFE707A8007808B080BDC0463FFFFF00C9
:105E940080B584B0029002980068C168A022914342
:105EA400C160FDF7D5F90190FFE702980068C0686A
:105EB400800600280DD4FFE7FDF7CAF90199401ABE
:105EC4000849884204D3FFE703A80321017004E0D2
:105ED400EBE703A800210170FFE703A8007804B0F2
:085EE40080BDC046E903000087
:105EEC0010B584B002900298002804D1FFE703A8F3
:105EFC000121017085E00298406A002801D1FFE77A
:105F0C00FFE702980021816202985D21405C002825
:105F1C0008D1FFE702985C2100224254029802F05B
:105F2C0089FDFFE702985D21022242540298006825
:105F3C0001684022914301600298C068334988424D
:105F4C0003D3FFE70020019003E001200003019040
:105F5C00FFE70298C0680F21090288420BD0FFE7C7
:105F6C000298C06807210902884204D0FFE7029812
:105F7C0000218162FFE70298006B00280FD1FFE738
:105F8C000298C0682149884204D3FFE70298022195
:105F9C00016303E0029801210163FFE7FFE7029828
:105FAC004168826811430269114342691143826955
:105FBC0001235C0222401143C2691143026A11435E
:105FCC00826A1143006801600298418B04221140DF
:105FDC00426A1143426B1143C2681143019A114347
:105FEC000068416002980068C169DA029143C1619E
:105FFC0002980021016602985D22835403A8017067
:10600C00FFE703A8007804B010BDC04601070000EC
:10601C00B0B58EB0129C1D460C900B910A9209A83B
:10602C0003800120039002A800210170FFE70C9867
:10603C005C21405C012804D1FFE70DA8022101700E
:10604C0000E20C985C2101224254FFE7FFE7FDF7C8
:10605C00FBF804900C985D21405C05A908700C9825
:10606C0040680690099808AA1080099807AA108021
:10607C000878012814D0FFE706984121890088424E
:10608C000AD1FFE70C988068002805D1FFE705A826
:10609C000078042804D0FFE702A802210170C3E1B4
:1060AC000B98002809D0FFE70A98002805D0FFE7D5
:1060BC0009A80088002804D1FFE702A8012101707B
:1060CC00B2E10C985D21405C042805D0FFE70C98E8
:1060DC005D2105224254FFE70C98002101660A98C5
:1060EC000C9A106409980C9A4623D05209980C9A71
:1060FC004423D0520B980C9A906309980C9AD08731
:10610C0009980C9A90870C98C1640C9801650C98AE
:10611C00C06807210902884205D8FFE707A8008854
:10612C00022808D3FFE70C9800684168012212038B
:10613C009143416007E00C9800684168012212030A
:10614C0011434160FFE70C9800680068402108404B
:10615C00402807D0FFE70C980068016840221143E3
:10616C000160FFE70C98C068B84988427ED3FFE70E
:10617C000C984068002805D0FFE708A80088012883
:10618C000ED1FFE70C98816B09880068C1600C98F0
:10619C00816B891C81630C98C18F491EC187FFE7F5
:1061AC00FFE70C98C08F01210028019107D1FFE770
:1061BC000C984621405A411E88410190FFE70198F6
:1061CC00C007002851D0FFE70C9800688068800752
:1061DC00002819D5FFE70C98C08F002814D0FFE7D2
:1061EC000398012810D1FFE70C98816B098800688F
:1061FC00C1600C98816B891C81630C98C18F491EFE
:10620C00C18700200390FFE70C9800688068C007E6
:10621C00002818D0FFE70C984621405A002812D0CD
:10622C00FFE70C980068C0680C99096C08800C9802
:10623C00016C891C01640C984621425A521E425230
:10624C0001200390FFE7FCF7FFFF0499401A129915
:10625C00884209D3FFE71298401C002804D0FFE7BE
:10626C0002A803210170DFE09BE7CDE00C984068A9
:10627C00002805D0FFE708A80088012822D1FFE7F5
:10628C000C98C08F02280ED3FFE70C98816B0988FD
:10629C000068C1600C98816B891C81630C98C18F5C
:1062AC00891EC1870DE00C98816B09780068017319
:1062BC000C98816B491C81630C98C18F491EC18756
:1062CC00FFE7FFE7FFE70C98C08F01210028009142
:1062DC0007D1FFE70C984621405A411E8841009097
:1062EC00FFE70098C007002800D18CE00C980068EC
:1062FC008068800700282DD5FFE70C98C08F0028F8
:10630C0028D0FFE70398012824D1FFE70C98C08F11
:10631C0002280ED3FFE70C98816B09880068C160D6
:10632C000C98816B891C81630C98C18F891EC18765
:10633C000DE00C98816B0978006801730C98816BE7
:10634C00491C81630C98C18F491EC187FFE700204F
:10635C000390FFE70C9800688068C00700283CD0C9
:10636C00FFE70C984621405A002836D0FFE70C98DE
:10637C004621405A02281DD3FFE70C980068C068DC
:10638C000C99096C08800C98016C891C01640C98A0
:10639C004621425A921E42520C98405A012808D863
:1063AC00FFE70C9800684168012212031143416019
:1063BC00FFE70FE00C980068007B0C99096C0870E3
:1063CC000C98016C491C01640C984621425A521ECF
:1063DC004252FFE701200390FFE7FCF735FF0499D9
:1063EC00401A1299884205D3FFE71298401C0028E6
:1063FC0004D1FFE71298002804D1FFE702A803217B
:10640C00017011E05FE7FFE70C981299049A07F00E
:10641C0002FF002807D0FFE702A8012101700C98A9
:10642C0020210166FFE7FFE70C985D210122425411
:10643C00FFE70C985C2100224254FFE702980DA95B
:10644C000870FFE70DA800780EB0B0BD0107000082
:10645C0080B584B00390029102980C28009028D843
:10646C000098C046784400794000874406222222D6
:10647C000D222222142222221B0003980068C168DC
:10648C0002221143C16015E003980068C168042220
:10649C001143C1600EE003980068C16808221143E3
:1064AC00C16007E003980068C16810221143C16005
:1064BC0000E0FFE7039800680299012207F0F6FE5E
:1064CC000398006880680B490840019001980628E1
:1064DC000DD0FFE7019801210904884207D0FFE79E
:1064EC00039800680168012211430160FFE7002056
:0864FC0004B080BD070001009F
:1065040080B582B0019001983D2102224254FFE7F8
:1065140001980068006A124908420FD1FFE7019808
:106524000068006A0F49084207D1FFE70198006834
:106534000168012291430160FFE7FFE7FFE701984B
:1065440008F0F4FB01983D2100224254FFE7019832
:106554003C2100224254FFE7002002B080BDC04627
:086564001111000044040000C5
:10656C0080B584B00390029102980C28019028D831
:10657C000198C046784400794000874406222222C4
:10658C000D222222142222221B0003980068C168CB
:10659C0002229143C16015E003980068C16804228F
:1065AC009143C1600EE003980068C16808229143D2
:1065BC00C16007E003980068C16810229143C16074
:1065CC0000E0FFE7039800680299002207F06EFED6
:1065DC00FFE703980068006A0B4908420FD1FFE7F8
:1065EC0003980068006A0949084207D1FFE703983D
:1065FC0000680168012291430160FFE7FFE7FFE7B4
:10660C00002004B080BDC0461111000044040000FD
:10661C0083B002900191029800680090029836496C
:10662C00884205D0FFE70298344988420AD1FFE737
:10663C0000987021884300900198406800990143AC
:10664C000091FFE702982C49884219D0FFE7029885
:10665C002A49884214D0FFE70298294988420FD072
:10666C00FFE70298274988420AD0FFE7029826499B
:10667C00884205D0FFE70298244988420BD1FFE7F6
:10668C00009803210902884300900198C068009982
:10669C0001430091FFE700988021884301994969E3
:1066AC00084300900098029908600198806802994C
:1066BC00C862019800680299886202980E49884263
:1066CC000FD0FFE702980F4988420AD0FFE70298E3
:1066DC000D49884205D0FFE702980C49884205D144
:1066EC00FFE70198006902990863FFE7029801210E
:1066FC00416103B07047C046002C014000040040CB
:10670C00002000400040014000440140004801408E
:10671C0087B006900591049203930698016A0122B2
:10672C00914301620698806902900698006A019074
:10673C0006982049884200920ED0FFE70698012166
:10674C001D4A9042009107D0FFE706981B4940185C
:10675C00414248410090FFE70098C007002809D04B
:10676C00FFE70298032188430290049802990143A1
:10677C00029104E00298012108430290FFE702987D
:10678C00F0218843029003980001C0B202990143A2
:10679C00029101980A2188430190059808400199BB
:1067AC000143019102980699886101980699086243
:1067BC0007B07047002C01400004004000C0FEBF31
:1067CC0080B582B0019001980068006902210840F0
:1067DC004008002828D0FFE701980068C068022113
:1067EC000840400800281ED0FFE7019800680221ED
:1067FC00C943016101980121017701980068806902
:10680C008007002804D0FFE7019804F06FFF06E032
:10681C00019808F003FC019808F0E4FCFFE70198EC
:10682C0000210177FFE7FFE7019800680069042168
:10683C0008408008002829D0FFE701980068C0684C
:10684C0004210840800800281FD0FFE70198006849
:10685C000421C94301610198022101770198006864
:10686C0080698005800F002804D0FFE7019804F0B0
:10687C003DFF06E0019808F0D1FB019808F0B2FC4E
:10688C00FFE7019800210177FFE7FFE70198006817
:10689C00006908210840C008002828D0FFE70198AB
:1068AC000068C06808210840C00800281ED0FFE717
:1068BC00019800680821C9430161019804210177FE
:1068CC0001980068C0698007002804D0FFE7019890
:1068DC0004F00CFF06E0019808F0A0FB019808F00A
:1068EC0081FCFFE7019800210177FFE7FFE70198A2
:1068FC0000680069102108400009002829D0FFE732
:10690C0001980068C06810210840000900281FD0B9
:10691C00FFE7019800681021C94301610198082123
:10692C00017701980068C0698005800F002804D0A9
:10693C00FFE7019804F0DAFE06E0019808F06EFB20
:10694C00019808F04FFCFFE7019800210177FFE761
:10695C00FFE7019800680069C007002811D0FFE725
:10696C0001980068C068C007002809D0FFE70198AB
:10697C0000680121C9430161019808F037FCFFE769
:10698C00FFE7019800680069C0B2C009002812D066
:10699C00FFE701980068C068C0B2C009002809D0A0
:1069AC00FFE7019800688021C9430161019808F054
:1069BC0071FCFFE7FFE701980068006901210902FB
:1069CC000840000A002811D0FFE701980068C06851
:1069DC00C0B2C009002808D0FFE701980068204920
:1069EC000161019808F0A6FCFFE7FFE70198006839
:1069FC000069402108408009002813D0FFE7019866
:106A0C000068C068402108408009002809D0FFE7D1
:106A1C00019800684021C9430161019808F002FB0C
:106A2C00FFE7FFE701980068006920210840400952
:106A3C00002813D0FFE701980068C06820210840A7
:106A4C004009002809D0FFE7019800682021C943BC
:106A5C000161019808F022FCFFE7FFE702B080BD5E
:046A6C00FFFEFFFF2B
:106A700080B586B0059005986021405A04A9088029
:106A8000059884214058222865D1FFE705986821A0
:106A9000405A02A90880FFE702A80088002837D0E2
:106AA000FFE705980068406A03A9088003980499E5
:106AB00008400599896D08700598816D491C8165AC
:106AC00005985E21425A521E42520598405A0028AB
:106AD00018D1FFE70598006801680122120291436E
:106AE0000160059800688168204A1140816005981E
:106AF00084212022425005980021C166059808F0A3
:106B000027FCFFE7FFE70298401E02A90880C3E7C1
:106B100005985E21405A01A908800888002819D0EC
:106B2000FFE701A8008805996822895A884211DA8E
:106B3000FFE7059800688168012212079143816090
:106B400005980949C166059800680168202211432B
:106B50000160FFE706E0059800688169082211439B
:106B60008161FFE706B080BD61E40008FEFFFFEF32
:106B700080B586B0059005986021405A03A9088029
:106B8000059884214058222867D1FFE7059868219D
:106B9000405A01A90880FFE701A80088002839D0E1
:106BA000FFE705980068406A02A908800598806D93
:106BB0000490029803990840049908800598816D13
:106BC000891C816505985E21425A521E42520598E1
:106BD000405A002818D1FFE7059800680168012293
:106BE000120291430160059800688168204A1140B3
:106BF0008160059884212022425005980021C166B9
:106C0000059808F0A5FBFFE7FFE70198401E01A9E2
:106C10000880C1E705985E21405A694608800888C7
:106C2000002819D0FFE76846008805996822895A2C
:106C3000884211DAFFE7059800688168012212078F
:106C40009143816005980949C1660598006801680B
:106C5000202211430160FFE706E005980068816982
:106C6000082211438161FFE706B080BDCBE3000835
:046C7000FEFFFFEF35
:106C740010B5FFB081B07F9000207B907AA9087096
:106C840079907F9881680269114342691143C06910
:106C940001437E917F98406E7E9901437E917F9857
:106CA40000680068604908407E9908437F99096834
:106CB40008607F98006840680321090388437F992E
:106CC400CA681043096848607F9880697E907F98FD
:106CD400006A7E9901437E917F98006880685349D9
:106CE40008407E9908437F99096888607F98006806
:106CF400C06A0F2188437F994A6A10430968C862B1
:106D0400FFE77F9800684A49884224D1FFE7494851
:106D14000068032108400328789017D87898C04663
:106D240078440079400087440109050D7CA80021BE
:106D340001700FE07CA8022101700BE07CA8042103
:106D4400017007E07CA80821017003E07CA81021F1
:106D54000170FFE749E07F9800683749884229D1EC
:106D6400FFE7344800680C2108400C2877901CD8B1
:106D74007798C04678440079400087440616161672
:106D84000E1616160A16161612007CA8002101709B
:106D94000FE07CA8022101700BE07CA804210170A3
:106DA40007E07CA80821017003E07CA81021017091
:106DB400FFE719E07F9800682049884204D1FFE783
:106DC4007CA8002101700EE07F9800681C4988426D
:106DD40004D1FFE77CA80021017003E07CA8102106
:106DE4000170FFE7FFE7FFE7FFE7FFE77F98C06970
:106DF4000121C903884200D09EE27CA800780828BB
:106E0400769000D975E276984000C0467844808830
:106E14004000874417006E02AE006E0242016E020B
:106E24006E026E02D901C046F369FFCFFFF4FF1171
:106E34000038014054100240004400400048004023
:106E4400004C0040FEF79EFC7F99496A002975902A
:106E540003D1FFE7012074907AE07F98406A01280B
:106E640003D1FFE7022073906FE07F98406A022805
:106E740003D1FFE70420729064E07F98406A0328FE
:106E840003D1FFE70620719059E07F98406A0428F7
:106E940003D1FFE7082070904EE07F98406A0528F0
:106EA40003D1FFE70A206F9043E07F98406A0628E9
:106EB40003D1FFE70C206E9038E07F98406A0728E2
:106EC40003D1FFE710206D902DE07F98406A0828D9
:106ED40003D1FFE720206C9022E07F98406A0928C4
:106EE40003D1FFE740206B9017E07F98406A0A289F
:106EF40003D1FFE780206A900CE07F98406A01216B
:106F04000A020B286991689201D069986890689880
:106F14006A90FFE76A986B90FFE76B986C90FFE7C5
:106F24006C986D90FFE76D986E90FFE76E986F9088
:106F3400FFE76F987090FFE770987190FFE7719882
:106F44007290FFE772987390FFE773987490FFE76D
:106F54007498759967900846679908F0F3FB4000A8
:106F64007F9949684A08801808F0ECFB80B27B904E
:106F7400C3E17F98406A002803D1FFE701206690AF
:106F84007AE07F98406A012803D1FFE702206590E8
:106F94006FE07F98406A022803D1FFE704206490E1
:106FA40064E07F98406A032803D1FFE706206390DA
:106FB40059E07F98406A042803D1FFE708206290D3
:106FC4004EE07F98406A052803D1FFE70A206190CC
:106FD40043E07F98406A062803D1FFE70C206090C5
:106FE40038E07F98406A072803D1FFE710205F90BC
:106FF4002DE07F98406A082803D1FFE720205E90A7
:1070040022E07F98406A092803D1FFE740205D9081
:1070140017E07F98406A0A2803D1FFE780205C903C
:107024000CE07F98406A01210A020B285B915A9276
:1070340001D05B985A905A985C90FFE75C985D90F9
:10704400FFE75D985E90FFE75E985F90FFE75F98CB
:107054006090FFE760986190FFE761986290FFE7B6
:1070640062986390FFE763986490FFE76498659083
:10707400FFE765986690FFE76698BA495990084615
:10708400599908F05FFB40007F9949684A088018C5
:1070940008F058FB80B27B902FE1FEF76DF97F99E1
:1070A400496A0029589003D1FFE7012057907AE0FC
:1070B4007F98406A012803D1FFE7022056906FE0D1
:1070C4007F98406A022803D1FFE70420559064E0CA
:1070D4007F98406A032803D1FFE70620549059E0C3
:1070E4007F98406A042803D1FFE7082053904EE0BC
:1070F4007F98406A052803D1FFE70A20529043E0B5
:107104007F98406A062803D1FFE70C20519038E0AD
:107114007F98406A072803D1FFE7102050902DE0A4
:107124007F98406A082803D1FFE720204F9022E08F
:107134007F98406A092803D1FFE740204E9017E06A
:107144007F98406A0A2803D1FFE780204D900CE025
:107154007F98406A01210A020B284C914B9201D07E
:107164004C984B904B984D90FFE74D984E90FFE70D
:107174004E984F90FFE74F985090FFE750985190EA
:10718400FFE751985290FFE752985390FFE75398C6
:107194005490FFE754985590FFE755985690FFE7B1
:1071A40056985790FFE7579858994A9008464A9935
:1071B40008F0C8FA40007F9949684A08801808F026
:1071C400C1FA80B27B9098E07F98406A002803D18E
:1071D400FFE7012049907AE07F98406A012803D1B3
:1071E400FFE7022048906FE07F98406A022803D1AD
:1071F400FFE70420479064E07F98406A032803D1A6
:10720400FFE70620469059E07F98406A042803D19E
:10721400FFE7082045904EE07F98406A052803D197
:10722400FFE70A20449043E07F98406A062803D190
:10723400FFE70C20439038E07F98406A072803D189
:10724400FFE7102042902DE07F98406A082803D180
:10725400FFE72020419022E07F98406A092803D16B
:10726400FFE74020409017E07F98406A0A2803D146
:10727400FFE780203F900CE07F98406A01210A02DA
:107284000B283E913D9201D03E983D903D983F9011
:10729400FFE73F984090FFE740984190FFE741980F
:1072A4004290FFE742984390FFE743984490FFE7FA
:1072B40044984590FFE745984690FFE746984790E5
:1072C400FFE747984890FFE748984990FFE74998B7
:1072D4000121C9033C9008463C9908F033FA400068
:1072E4007F9949684A08801808F02CFA80B27B908C
:1072F40003E07AA801210170FFE77B98102816D3D8
:10730400FFE77BA84088002811D1FFE77B980F2175
:1073140088437DA908807B980E22104040087D9AFE
:1073240002430A8008887F990968C86003E07AA844
:1073340001210170FFE781E27CA8007808283B90D6
:1073440000D964E23B984000784480884000874438
:107354000B005E02A1005E0234015E025E025E0268
:10736400CA01C0460024F400FEF70CFA7F99496A6A
:1073740000293A9003D1FFE7012039907AE07F9801
:10738400406A012803D1FFE7022038906FE07F981C
:10739400406A022803D1FFE70420379064E07F9815
:1073A400406A032803D1FFE70620369059E07F980E
:1073B400406A042803D1FFE7082035904EE07F9807
:1073C400406A052803D1FFE70A20349043E07F9800
:1073D400406A062803D1FFE70C20339038E07F98F9
:1073E400406A072803D1FFE7102032902DE07F98F0
:1073F400406A082803D1FFE72020319022E07F98DB
:10740400406A092803D1FFE74020309017E07F98B5
:10741400406A0A2803D1FFE780202F900CE07F9870
:10742400406A01210A020B282E912D9201D02E9838
:107434002D902D982F90FFE72F983090FFE73098EC
:107444003190FFE731983290FFE732983390FFE7AD
:1074540033983490FFE734983590FFE735983690A9
:10746400FFE736983790FFE737983890FFE738986A
:107474003990FFE739983A992C9008462C9908F0EE
:1074840061F97F9949684A08801808F05BF980B26D
:107494007B90C0E17F98406A002803D1FFE7012078
:1074A4002B907AE07F98406A012803D1FFE70220FD
:1074B4002A906FE07F98406A022803D1FFE70420F6
:1074C400299064E07F98406A032803D1FFE70620EF
:1074D400289059E07F98406A042803D1FFE70820E8
:1074E40027904EE07F98406A052803D1FFE70A20E1
:1074F400269043E07F98406A062803D1FFE70C20DA
:10750400259038E07F98406A072803D1FFE71020D0
:1075140024902DE07F98406A082803D1FFE72020BB
:10752400239022E07F98406A092803D1FFE7402096
:10753400229017E07F98406A0A2803D1FFE7802051
:1075440021900CE07F98406A01210A020B282091C7
:107554001F9201D020981F901F982190FFE7219837
:107564002290FFE722982390FFE723982490FFE7D7
:1075740024982590FFE725982690FFE726982790E2
:10758400FFE727982890FFE728982990FFE7299894
:107594002A90FFE72A982B90FFE72B98B0491E907A
:1075A40008461E9908F0CEF87F9949684A08801861
:1075B40008F0C8F880B27B902DE1FDF7DDFE7F99DD
:1075C400496A00291D9003D1FFE701201C907AE04D
:1075D4007F98406A012803D1FFE702201B906FE0E7
:1075E4007F98406A022803D1FFE704201A9064E0E0
:1075F4007F98406A032803D1FFE70620199059E0D9
:107604007F98406A042803D1FFE7082018904EE0D1
:107614007F98406A052803D1FFE70A20179043E0CA
:107624007F98406A062803D1FFE70C20169038E0C3
:107634007F98406A072803D1FFE7102015902DE0BA
:107644007F98406A082803D1FFE72020149022E0A5
:107654007F98406A092803D1FFE74020139017E080
:107664007F98406A0A2803D1FFE7802012900CE03B
:107674007F98406A01210A020B281191109201D0CF
:107684001198109010981290FFE712981390FFE74A
:1076940013981490FFE714981590FFE71598169027
:1076A400FFE716981790FFE717981890FFE71898C8
:1076B4001990FFE719981A90FFE71A981B90FFE7B3
:1076C4001B981C90FFE71C981D990F9008460F9972
:1076D40008F038F87F9949684A08801808F032F8A9
:1076E40080B27B9097E07F98406A002803D1FFE73F
:1076F40001200E907AE07F98406A012803D1FFE7C9
:1077040002200D906FE07F98406A022803D1FFE7C2
:1077140004200C9064E07F98406A032803D1FFE7BB
:1077240006200B9059E07F98406A042803D1FFE7B4
:1077340008200A904EE07F98406A052803D1FFE7AD
:107744000A20099043E07F98406A062803D1FFE7A6
:107754000C20089038E07F98406A072803D1FFE79F
:10776400102007902DE07F98406A082803D1FFE796
:107774002020069022E07F98406A092803D1FFE781
:107784004020059017E07F98406A0A2803D1FFE75C
:10779400802004900CE07F98406A01210A020B28A3
:1077A4000391029201D00398029002980490FFE79B
:1077B40004980590FFE705980690FFE70698079060
:1077C400FFE707980890FFE708980990FFE70998F2
:1077D4000A90FFE70A980B90FFE70B980C90FFE7DD
:1077E4000C980D90FFE70D980E90FFE70E9801217D
:1077F400C90301900846019907F0A4FF7F994968DD
:107804004A08801807F09EFF80B27B9003E07AA8B4
:1078140001210170FFE77B9810280AD3FFE77BA8BA
:107824004088002805D1FFE77B987F990968C860E4
:1078340003E07AA801210170FFE7FFE77F986A213E
:10784400012242527F98682142527F980021C166EA
:107854007F9801677AA800787FB001B010BDC04658
:047864000024F40008
:1078680084B01346029001916846028002988021F4
:107878004058202800D097E00198002805D0FFE75D
:1078880068460088002804D1FFE703A80121017099
:107898008EE00298806801210903884210D1FFE731
:1078A8000298006900280BD1FFE701A80078C007FB
:1078B800002804D0FFE703A80121017078E0FFE762
:1078C800FFE702987C21405C012804D1FFE703A868
:1078D800022101706CE002987C2101224254FFE7EA
:1078E800FFE7019802990865009802995422885286
:1078F800009802995622885202980021016702983E
:107908008822815002988021212242500298406E9C
:1079180001214907884222D1FFE7029880680121A6
:107928000903884209D1FFE702980069002804D1B9
:10793800FFE702982349016703E00298204901679D
:10794800FFE7FFE702987C2100224254FFE70298F4
:10795800006881680122D2051143816020E0029805
:10796800806801210903884209D1FFE7029800696C
:10797800002804D1FFE702981049016703E0029844
:107988000D490167FFE7FFE702987C210022425476
:10799800FFE7029800680168802211430160FFE751
:1079A80003A80021017003E003A802210170FFE78A
:1079B80003A8007804B070474DE60008717A000803
:0879C800B1F20008D1790008BA
:1079D00083B00290029880214058212843D1FFE7CC
:1079E00002986A21405A69460880FFE76846008885
:1079F000002837D0FFE702985621405A00280ED1C0
:107A0000FFE70298006881680122D20591438160F6
:107A100002980068016840221143016022E0029848
:107A20000068C0690006002814D5FFE70298006DC1
:107A30000190019800880D49084002990968886200
:107A40000298016D891C016502985621425A521E06
:107A5000425200E0FFE7FFE7FFE70098401E69465B
:107A60000880C3E7FFE703B07047C046FF0100008E
:107A700082B00190019880214058212828D1FFE749
:107A800001985621405A00280DD1FFE7019800685F
:107A900001688022914301600198006801684022DA
:107AA0001143016013E00198006D00900098008878
:107AB000084908400199096888620198016D891C8C
:107AC000016501985621425A521E4252FFE7FFE7D4
:087AD00002B07047FF01000045
:107AD80084B013460290019168460280029884217E
:107AE8004058202800D0F8E00198002805D0FFE78A
:107AF80068460088002804D1FFE703A80121017027
:107B0800EFE00298806801210903884210D1FFE75D
:107B18000298006900280BD1FFE701A80078C00788
:107B2800002804D0FFE703A801210170D9E0FFE78E
:107B3800FFE702987C21405C012804D1FFE703A8F5
:107B480002210170CDE002987C2101224254FFE716
:107B5800FFE7019802998865009802995C2288528B
:107B6800009802995E22885202980021C166FFE7B8
:107B78000298806801210903884210D1FFE7029822
:107B88000069002805D1FFE702986021574A425250
:107B980004E002986021FF224252FFE732E0029897
:107BA8008068002810D1FFE702980069002805D1F5
:107BB800FFE702986021FF22425204E00298602108
:107BC8007F224252FFE71CE00298806801210907E2
:107BD800884210D1FFE702980069002805D1FFE725
:107BE800029860217F22425204E0029860213F22DD
:107BF8004252FFE704E00298602100224252FFE768
:107C0800FFE7FFE7FFE70298882100224250029829
:107C1800842122224250029800688168012211437F
:107C280081600298406E5107884230D1FFE768466C
:107C3800008802996822895A884228DBFFE702985F
:107C4800806801210903884209D1FFE70298006989
:107C5800002804D1FFE702982849C16603E002988A
:107C68002549C166FFE7FFE702987C2100224254BC
:107C7800FFE70298006801680122130219430160B6
:107C880002980068816812071143816021E0029818
:107C9800806801210903884209D1FFE70298006939
:107CA800002804D1FFE702981249C16603E0029850
:107CB8000F49C166FFE7FFE702987C210022425482
:107CC800FFE7029800680168092252011143016028
:107CD800FFE703A80021017003E003A80221017057
:107CE800FFE703A8007804B07047C046FF01000012
:107CF80061E40008CBE30008716A0008716B0008B2
:107D080080B584B002900298882100224250FBF787
:107D18009DFA01900298006800680007002811D5B4
:107D2800FFE70298019B1E490091012149050022A5
:107D380007F062FA002804D0FFE703A803210170C6
:107D480029E0FFE70298006800684007002811D57D
:107D5800FFE70298019B1249009101218905002241
:107D680007F04AFA002804D0FFE703A803210170AE
:107D780011E0FFE7029880212022425002988421D6
:107D88004250FFE702987C2100224254FFE703A8F3
:107D980000210170FFE703A8007804B080BDC04649
:047DA800FFFFFF01D9
:107DAC0080B584B000200390029001905649574A48
:107DBC000A60072292044A608860C8600122530559
:107DCC000B6108234B61087648768A76CB612023B9
:107DDC00C854486288622C23CA5413030B630523CE
:107DEC004B638B633C23CA540C220A64486488643A
:107DFC00C8640846FBF75CFA002803D0FFE706F0DE
:107E0C0089FCFFE7012001900020029007200390DD
:107E1C003D4801A9FBF76EFD002803D0FFE706F0F3
:107E2C0079FCFFE73A480190042002900720039068
:107E3C00354801A9FBF75EFD002803D0FFE706F0EB
:107E4C0069FCFFE73348019008200290072003905B
:107E5C002D4801A9FBF74EFD002803D0FFE706F0E3
:107E6C0059FCFFE72C4801900C200290072003904E
:107E7C00254801A9FBF73EFD002803D0FFE706F0DB
:107E8C0049FCFFE725480190102002900720039041
:107E9C001D4801A9FBF72EFD002803D0FFE706F0D3
:107EAC0039FCFFE71E480190142002900720039034
:107EBC00154801A9FBF71EFD002803D0FFE706F0CB
:107ECC0029FCFFE717480190182002900720039027
:107EDC000D4801A9FBF70EFD002803D0FFE706F0C3
:107EEC0019FCFFE7104801901C200290072003901A
:107EFC00054801A9FBF7FEFC002803D0FFE706F0BC
:107F0C0009FCFFE704B080BDE00B00200024014019
:107F1C0002000004040000080001002000020024FC
:0C7F2C0000040028001000B0002000B489
:107F3800B0B594B0139000201290119010900F904B
:107F48000E90139800684F49884200D098E0FFE7E8
:107F58004D48016801221205114301600068104074
:107F68000D900D98FFE7FFE748480168012211438B
:107F78000160006810400C900C98FFE7FFE7434849
:107F88000168022211430160006810400B900B98B1
:107F9800FFE701200E9003210F9100221092052384
:107FA8001C070EAD0A9020460991294608920793AE
:107FB80006940595FCF744FB02200E9009990F9151
:107FC800089A1092069B049018460599FCF738FB0E
:107FD80004200E9009990F91089A1092069B03901D
:107FE80018460599FCF72CFB0A980E9009990F91F1
:107FF800089A1092264B184605990293FCF720FB25
:1080080004980E9009990F91089A10920298059970
:10801800FCF716FB03980E9009990F91089A109295
:1080280002980599FCF70CFB1A481B49016007994F
:108038004160089A8260C260802303610A9B1C0227
:108048004461DC0284612024C4610262FCF7ACF85C
:10805800002803D0FFE706F05FFBFFE7FFE7139870
:108068000C49016513988862FFE70C2000210190F4
:108078000091009A05F0D5FF019806F043FEFFE74E
:1080880014B0B0BD0024014040100240341002403A
:0C80980000040050A80C0020080002406A
:1080A40080B58EB000200C900B900A900990089037
:1080B4000790069006A8FCF755FC06200690BB2006
:1080C4000A90072000060B90052000060C90FCF790
:1080D40041FA002804D0FFE71E4807F029FAFFE719
:1080E400FCF712FA002804D0FFE71B4807F020FA37
:1080F400FFE71A4807F01CFA06A905900846FCF7A2
:10810400FBFC00280AD0FFE7184807F011FA049096
:10811400FCF746FA0DA900220A7017E0FCF740FAB2
:108124000F490390084607F003FA0290FCF750FA4F
:108134000C490190084607F0FBF90B4900900846EA
:1081440007F0F6F90DA901220A70FFE70DA80078DF
:108154000EB080BDFCF8000810F9000827F90008EB
:108164004EF9000867F9000876F9000838F90008A4
:1081740081B0009002480121016001B07047C046FF
:04818400C40D002006
:1081880080B590B000200F900E900D900C900B9041
:10819800FFE7464801680222114301600068104069
:1081A8000A900A98FFE7FFE7404801680422114354
:1081B80001600068104009900998FFE7FFE73B4815
:1081C8000168202211430160006810400890089857
:1081D800FFE7FFE7354801680122114301600068A5
:1081E800104007900798FFE7052000073049002254
:1081F80006900591049205F0AAFF012001022D4A7C
:10820800039010460291049B01921A4605F09FFFC5
:10821800039841020B9128490C910D900BA90198E4
:108228000091FCF70DFA05980B9003990C91049AAC
:108238000D920E9206980099FCF702FA40200B90D6
:1082480004980C9003990D911C480099FCF7F8F9D3
:1082580002980B9003990C91049A0D920E92019832
:108268000099FCF7EDF9039801030B9104990C911F
:108278000D900E9106980099FCF7E2F910200B90EA
:1082880003980C900D9004990E9101980099FCF7B1
:10829800D7F920200B9003980C900D9004990E911B
:1082A80001980099FCF7CCF910B080BD3410024059
:1082B800389F000000040050000021100008005002
:1082C80080B588B000200790069005900490039030
:1082D8000290019001A8FCF743FB0598AA2807D152
:1082E800FFE7134807F022F9694600220A7017E0F1
:1082F8000598BB2807D1FFE70C4807F017F969462E
:1083080001220A700BE00598CC2807D1FFE7064840
:1083180007F00CF9694602220A70FFE7FFE7FFE75A
:108328006846007808B080BD77FA00085BFA000854
:048338003FFA000800
:10833C0080B59EB011A83421059007F083FA002077
:10834C0010900F900E900D900C900B900A9009903D
:10835C0008900790069001214A0204901046039160
:10836C00FDF7CAF90290FCF79FFC2048016818221F
:10837C0011430160FCF78EFC0620119003981390BA
:10838C0001021491049915914022169218910598A6
:10839C00FCF79CFC002803D0FFE706F0BBF9FFE7D5
:1083AC0007200D9000200E900F9010900DA90190B9
:1083BC0008460199FDF76AF8002803D0FFE706F09C
:1083CC00A9F9FFE70A480690002007900B900120BE
:1083DC0000020C9006A8FDF769FA002803D0FFE70D
:1083EC0006F098F9FFE71EB080BDC0465C10024055
:0483FC00014002003A
:1084000080B59AB0014618AA1070002017901690F7
:108410001590149013901290119011A810910F9232
:10842000FCF7A2FA0F980178C90700294CD0FFE7A2
:108430005C4807F07FF81599AA2940D1FFE7022090
:108440001190BB201590FCF787F8002804D0FFE7B7
:10845000534807F06FF8FFE7FCF758F8002804D0FE
:10846000FFE74E4807F066F8FFE7504807F062F86C
:1084700011A90E900846FCF741FB00280AD0FFE73F
:108480004C4807F057F80D90FCF78CF819A900221A
:108490000A7071E0FCF786F83C490C90084607F03A
:1084A00049F80B90FCF796F839490A90084607F00E
:1084B00041F83F490990084607F03CF803E03A4884
:1084C00007F038F8FFE753E01598BB284FD1FFE7D6
:1084D00002201190AA201590FCF73EF8002807D042
:1084E000FFE72F4807F026F819A900220A7043E099
:1084F000234807F01FF80890FCF708F8002807D079
:10850000FFE7264807F016F819A900220A7033E0A1
:108510001C4807F00FF811A907900846FCF7EEFA7F
:1085200000280BD0FFE7FCF73DF81B4906900846F2
:1085300007F000F819A900220A701DE0124806F0A1
:10854000F9FF0590FCF72EF810490490084606F054
:10855000F1FF0390FCF73EF80D490290084606F043
:10856000E9FF0C490190084606F0E4FFFFE7FFE74A
:1085700019A801210170FFE719A800781AB080BD81
:10858000B5F90008C8F9000800FA00084EF900081B
:1085900067F900081DFA0008DEF9000810F9000864
:1085A000FCF80008DBF8000897F9000827F9000834
:0885B00076F9000838F9000813
:1085B800BFF34F8F034804490160BFF34F8FFFE7B4
:0C85C80000BFFDE70CED00E00400FA0528
:1085D40010B59CB010A80021C162C16181614161E4
:1085E40012AA117011AA1170BF4A7D239B00138037
:1085F40001231381518103219181D907E824115169
:10860400EC21BA4C5450D903D023D152D221B84BC7
:108614005352DC21B74C5450E02153500E90FFF7D5
:1086240051FE002801D1FFE7FFE7FAF717FE0D908E
:10863400FFF782FEFFF746FEAF490C90084606F0AE
:1086440077FF0B9003F0C4F902F0B2FF03F0E4F8F3
:10865400FFF798FD00F0D8FB00F0ACF9FFF7A4FB9E
:1086640000F028FA01F0CCF9002809D0FFE7A3486C
:1086740006F05EFF9C490A90084601F02BFAFFE7DA
:108684009F4806F055FF98490990084601F09EF866
:108694009C49402208900846114605F073FD0028C5
:1086A40009D1FFE7984806F043FF8F490790084631
:1086B40001F016FBFFE78C480169828A934B944CC6
:1086C40006901846234606F0A1FF069801F0E2FE44
:1086D40090480590FBF764FB8F490822059B0490A2
:1086E4001846FAF7BFFF039000F026F900F09EFD4C
:1086F4008A4806F01DFF029002F0AEFAFFE78848B0
:10870400006801281CD1FFE78548002101608248E8
:10871400C1680190084601F0FFFE0198006801F06D
:108724002FFF0198806901F0FBFC0198406901F07A
:108734004DFF019840680199896801F021FDFFE728
:10874400FAF786FD0E994862486A8A6A801A0862B6
:10875400486A8862086ACA691018C861086A8A691E
:10876400101888616F48026812680F231A4012AB10
:108774001A7000684068086011A800781A7890425E
:1087840011D0FFE70E98816811AA1170052108071E
:108794000121890205F00DFD01F068FD02F03AF9AE
:1087A40001F0AAFFFFE75048408B002800D184E085
:1087B40056482621405C00287DD1FFE74A48408B7B
:1087C4000128009039D0FFE7009802283AD0FFE74B
:1087D400009803283AD0FFE7009804283AD0FFE72E
:1087E400009806283FD0FFE7009807283ED0FFE70F
:1087F400009808283ED0FFE7009809283ED0FFE7FC
:1088040000980A283DD0FFE700980B283DD0FFE7E9
:108814004548009981423BD0FFE744480099814292
:108824003AD0FFE7FD2080000099814238D0FFE76D
:108834003F480099814211D035E02B48002101F0D6
:1088440015FB34E0284801F045F930E0264801F0F2
:1088540047FA2CE0244800F0B9FF28E0224801211F
:1088640001F004FB23E0FFF7A5FE20E01E4806F01C
:108874008DFD1CE01C4800F07FFA18E000F0A0FA1F
:1088840015E0194800F00AFB11E000F003FC0EE0CB
:108894000020FFF7B3FD0AE00120FFF7AFFD06E07B
:1088A400FFF7FEFB03E0234806F042FEFFE70E4815
:1088B4000021418300E0FFE7FFE7144806F09EFE35
:1088C400002810D0FFE7114802F088FB022804D1E9
:1088D400FFE70E4805F0C3FF04E00D48842122227F
:1088E4004250FFE7FFE70AE7C0080020FFFFFF7FD1
:1088F400FF7F00000080FFFF74F8000887F800087D
:1089040098F8000800080050A8F800088C0400201B
:10891400D8090020E00B0020700D0020BCF80008EE
:10892400C40D0020440D0020F2030000F3030000F6
:08893400D2040000CAF800089B
:10893C0080B584B001200102094A039010460291CF
:10894C00039B01921A4605F000FC7D208000FAF78B
:10895C0011FC00220198029905F0F7FB04B080BDD0
:04896C0000040050B3
:1089700082B00190019800680C49884213D1FFE74A
:10898000FFE70B4801680122920211430160006871
:10899000104000900098FFE7064801680122D203CA
:1089A00011430160FFE702B07047C0460028004055
:0889B0003C1002405C10024083
:1089B80080B51048104901604121890041600021BB
:1089C800816007221302C3600161012343619B0494
:1089D80083610823C361016241628162C2620163EB
:1089E8004163FDF77FFA002803D0FFE705F094FE06
:0C89F800FFE780BD440C0020003001406F
:108A040082B0FFE70B48016801221143016000684E
:108A1400104001900198FFE7FFE707480168012231
:108A24001207114301600068104000900098FFE7AE
:0C8A340002B07047401002403C100240AD
:108A400080B588B0079000200690059004900390B0
:108A50000290079800681549884225D1FFE7FFE793
:108A6000134801680122120311430160006810409D
:108A700001900198FFE7FFE70E48016801221143CA
:108A800001600068104000900098FFE7F02002901D
:108A90000220039000200490059006900520000716
:108AA00002A9FBF7D1FDFFE708B080BD003001400F
:088AB0004010024034100240A6
:108AB80080B58AB00020099008900790069005902C
:108AC80004902449244A0A6088607F22CA60FF22F1
:108AD8000A6148618861C861012292070A62486296
:108AE8000846FDF70BF8002803D0FFE705F014FE51
:108AF800FFE705A8022101700021417081700691ED
:108B08000891099113490122039008460399FDF73A
:108B180077F8002803D0FFE705F0FEFDFFE704A87B
:108B28000121017004224270162282701822C2703C
:108B3800084A02901046029A01911146019AFDF7DF
:108B48000DF9002803D0FFE705F0E6FDFFE70AB0BE
:0C8B580080BDC046440D002000280040F5
:108B640080B5024802F0B6FB80BDC046D80900209B
:108B740080B50248FBF726FA80BDC046A80C002049
:108B840080B50248FDF720FE80BDC046040D0020DC
:108B9400014802490160704708ED00E00030000818
:108BA40080B588B03E4800683821084020280190EC
:108BB40000D954E00198C0467844007940008744C5
:108BC4004D4E4E4E4E4E4E4E104E4E4E4E4E4E4E00
:108BD4001E4E4E4E4E4E4E4E144E4E4E4E4E4E4E1B
:108BE400190033483149016049E031487D210902C7
:108BF400016044E02E480121C90301603FE0294897
:108C040001680322114004910068702108400009A2
:108C1400401C03900498032806D1FFE703992348D6
:108C240006F090FD069005E003991F4806F08AFDC2
:108C34000690FFE706981B490A687F231B021A4027
:108C4400120A424306920868400F401C0590069899
:108C5400059906F077FD1649086010E0FFE715480E
:108C640000680721C9020840C00A0121814002911D
:108C740002990D4806F066FD0D490860FFE70848B3
:108C840000680F210902084080090B490858079021
:108C9400079807490A68C2400A6008B080BDC04608
:108CA400081002400C1002400024F40000127A0064
:0C8CB40088000020001002409CD900083D
:108CC00080B58EB00D9000200C900B900A9009900A
:108CD00008900D9800682549884244D1FFE7FFE7D6
:108CE000234801680122920311430160006810408B
:108CF00007900798FFE7FFE71E480168022211432B
:108D000001600068104006900698FFE70820089070
:108D10000220099000210A910B9104220C92164A1C
:108D200008AB059010460491194603920293FBF795
:108D30008BFCC02008900598099001210A91049AA3
:108D40000A920B920C920398029B01911946FBF731
:108D50007BFC1B2000900199049A05F066F90098AD
:108D600005F0D4FFFFE70EB080BDC04600380140DB
:0C8D70004010024034100240000400508B
:108D7C0080B586B005900598D42141588422815045
:108D8C000598815880228058081A04900948006878
:108D9C00039003987D21C900414304980190084633
:108DAC00019906F0ADFC0290029805998822885032
:088DBC0006B080BDE80D0020A7
:108DC40080B584B00E48CC21415A8C228152815EF8
:108DD4007E22825E891A03910A49096802910299E6
:108DE4007D22D2004A4303990090104606F08CFC81
:108DF400019001989021009A505004B080BDC04663
:088E0400C0080020E00D002071
:108E0C0080B582B0FFE70A48016801221143016076
:108E1C000068104001900198FFE709200121002211
:108E2C00009005F0FCF8009805F06AFF02B080BDD8
:048E3C0038100240A8
:108E400010B586B0059004A80021817012490180F8
:108E500005990A2200920223039008460399039C75
:108E600002922246FDF7DAF82621039A117005993D
:108E7000029B00930323019008461146FDF7CEF8AC
:108E800003998A78102A05D0FFE7044806F052FBC0
:108E9000FFE7FEE706B010BD4610000004FE000824
:108EA000B0B596B015904C4806F044FB15999C223D
:108EB0008958002904D1FFE7524806F03BFB89E0BE
:108EC00015989C214058119102F0AEFE0022434BB0
:108ED00010920F9302F0A8FD414A136854680E9255
:108EE0001A46234602F0A0FD13911290129813998E
:108EF0003C4A109B0D921A460D9B05F022FD03F093
:108F000017F91599942288501598CE21415A982323
:108F1000C1521598CC21415A9A2401530E984168A8
:108F2000056831480C922A460B930B460A9406F0CA
:108F300001FB1599119A89580990084602F074FEB0
:108F4000109A0F9B02F070FD284A08901046089A6C
:108F50000B4606F0EFFA15990B9A895E07900846C2
:108F600002F062FE224A109B06921A46069B02F00D
:108F70005BFD204A05901046059A0B4606F0DAFA8A
:108F800015990A9A895E0490084602F04DFE109ADF
:108F9000069B02F049FD184A03901046039A0B46BF
:108FA00006F0C8FA15990C9A89580290084602F002
:108FB0003BFE109A0D9B05F0C4FC104A0190104630
:108FC000019A0B4606F0B6FA0D490090084606F0E5
:108FD000B1FAFFE716B0B0BD78FC000800408F4042
:108FE000C80D002080842E41E4FC000801FD00082B
:108FF0000000594010FD00081BFD000825FD000879
:0890000039FD00088AFC00089C
:1090080070B58CB00A460B900AA8017009A92323F1
:109018000B700B9C0A2500950326089020460791A3
:10902800079C069222460593334604950396FCF75F
:10903800F1FF07998A78EF231A400A9B1A434A706E
:1090480043220A700B9A049B009302230290104655
:10905800079AFCF7DFFF0599079A11700B9B049C90
:109068000094019018461146039BFCF7D3FF07991B
:109078008A78089B1C782240A24205D0FFE7034863
:1090880006F054FAFFE7FEE70CB070BD29FE0008B1
:1090980010B59AB0574806F049FA5749CE228B5A6C
:1090A800A0240B530B5F169018461591149202F0EA
:1090B800B7FD0022514B1392129302F0B1FC504AB3
:1090C80011901046119A0B4606F030FA1599149A29
:1090D8008B5E98240C5F1B1B1793179B10901846E8
:1090E80002F09EFD139A129B02F09AFC454A0F90DB
:1090F80010460F9A0B4606F019FA43490A684B685E
:10910800199318924B680A6840490E90084606F071
:109118000DFA9C21159A53580D9018460C9102F09F
:109128007FFD3B4A139B0B921A460B9B02F078FC7F
:10913800384A0A9010460A9A0B4606F0F7F915992C
:109148000C9A8B580990184602F06AFD139A0B9BEB
:1091580002F066FC189A199B02F062FC19911890AB
:10916800189819992C4A139B08921A46089B03F0E1
:1091780033F81991189018981999179A079010466A
:10918800069102F04DFD079A05901046069B049142
:109198001946059A049B02F043FC199118901898F7
:1091A80019991E4A139B03921A46039B05F0C5FBA7
:1091B80002F0BAFFA421159A5050505802F030FD21
:1091C800139A039B02F02CFC139A129B05F0B5FB33
:1091D800139A089B02F04CFD114A02901046029A1D
:1091E8000B4606F0A3F90F490190084606F09EF9D0
:1091F8001AB010BD4FFD0008C008002000005940FB
:1092080066FD000876FD0008D00D002085FD0008E9
:1092180000408F40B8FD00080000F03F65CDCD410B
:08922800C2FD0008E5FD00088D
:1092300010B58EB04248017A427A120251180BAA38
:10924000118101794279120251188279C3791B0286
:109250009A18120451180C91017842781202511890
:109260008278C07800028018000440180B903548BE
:109270000021017005221207082301240A901046DC
:1092800009911946089222460793069404F063FF59
:1092900096200590F9F774FF2B4810210490039154
:1092A000099A04F058FF0598F9F76AFF04980399A2
:1092B000069A04F050FF0598F9F762FF2020049900
:1092C000029008460299099A04F045FF0598F9F7BB
:1092D00057FF04980299069A04F03DFF0598F9F7A4
:1092E0004FFF08980799099A04F035FF07200221DB
:1092F0000190099A04F099FE019805F007FD1348C2
:109300000090FFF79DFD0598F9F73AFF0098029944
:1093100000F09CF800980999FFF776FE00980299F2
:1093200000F016F83421009800F05AF80598F9F783
:1093300027FF03200A99087006F042F80EB010BD0E
:10934000A5FE00082A0E002000040050440C002056
:1093500070B58CB00A460B900AA8017009A92323A6
:109360000B700B9C0A250095032608902046079158
:10937000079C069222460593334604950396FCF714
:109380004DFE07998A789F231A400A9B1A434A7018
:1093900043220A700B9A049B00930223029010460A
:1093A000079AFCF73BFE0599079A11700B9B049CEA
:1093B0000094019018461146039BFCF72FFE079975
:1093C0008A78089B1C782240A24205D0FFE7034818
:1093D00006F0B0F8FFE7FEE70CB070BD4BFE0008EA
:1093E000B0B58AB00A46099008A8017007A95123B0
:1093F0000B70089B4B7000238B70099B0A24009410
:109400000225069018460591059B04921A462B46A4
:109410000394FCF703FE3121059A11700999039B0F
:1094200000930323029008461146FCF7F7FD0599C7
:109430008A78069B1C78A24204D0FFE7024806F017
:0C94400079F8FFE70AB0B0BD67FE000835
:10944C0070B58CB00A460B900AA8017009A92223AA
:10945C000B700B9C0A25009503260890204607915B
:10946C00079C069222460593334604950396FCF717
:10947C00CFFD07998A7807231A400A9B1A434A7032
:10948C0042220A700B9A049B00930223029010460E
:10949C00079AFCF7BDFD0599079A11700B9B049C6C
:1094AC000094019018461146039BFCF7B1FD0799F7
:1094BC008A78089B1C782240A24205D0FFE703481B
:1094CC0006F032F8FFE7FEE70CB070BD3BFC00087D
:1094DC0010B588B02448017A427A1202511804AAB5
:1094EC001181017943791B0259188379C4792402BB
:1094FC00E3181B0459180591017843781B0259187D
:10950C008378C0780002C0180004401804900A2028
:10951C0000901648052311460292FCF779FD07A925
:10952C000022CA70029A93788B70D3784B70059B8B
:10953C000B700799C90D002907D0FFE707980C4954
:10954C00401807900798039008E00798C00D002872
:10955C0003D1FFE707980390FFE7FFE7039800F0BC
:10956C0009F808B010BDC04631FC0008440C0020BE
:04957C00010000FFEB
:10958000F0B5A7B0269082480168CA0F8A18521019
:10959000891A016026990268511801600068C10F9C
:1095A00040184010259025987A492122D2008850F1
:1095B00025988A6F801A784A1060D4200858802332
:1095C000CB58C01A249024988823CB58434318467C
:1095D0001791169202F028FB0022704B15921493FB
:1095E00002F022FA02F0A4FD23902398432189007F
:1095F000179A505016980168239BC91A684B196036
:10960000CC21515E7E24145F081B139302F00CFBE7
:1096100021912090209821999022179B9A5812907E
:109620001046119102F000FB129A10901046119B07
:109630000F911946109A0F9B05F083F9159A149B08
:1096400002F0F2F902F074FD1F90139801681F9A5E
:10965000891A544A1160106802F0E6FA524B159AC2
:1096600005F06FF9514B159A05F06BF9504B159AAF
:1096700002F0DAF94F4A5160106010685168942284
:10968000179B9A580E9010460D9102F0CDFA4A4B56
:10969000159A02F0C9F90E9A0C9010460D9B0B9189
:1096A00019460C9A0B9B05F04CF9444A5160106026
:1096B000CE201799085E9823CB5EC01A0A9202F05A
:1096C000B3FA1D911C90A4201799085802F0ACFA27
:1096D0003B4B159A02F0A8F91B911A901C981D9902
:1096E0001A9A1B9B05F02DF9364B159A02F0C4FA15
:1096F000199118900A9800680A994968189A199B54
:1097000005F01FF9304A516010600A9843680168FB
:1097100014685568189E199F1C9809901D9805900B
:10972000099804900397029601950094274808929F
:109730000A4605F0FFFE08990A6849680790104636
:10974000159A149B05F0FDF803F0FEF902F0F0FC09
:10975000E421179A50505058E8215158884206DDAC
:10976000FFE70C48E4214158E8228150FFE709480F
:10977000E4214158EC228058814206DAFFE705488F
:10978000E4214158EC228150FFE7002027B0F0BDD2
:10979000E40D0020C0080020E80D002000408F40AC
:1097A000E00D0020EC0D00200000044000406F4060
:1097B00000006041C80D002080842E41D00D0020A3
:1097C00065CDCD410000F03FD80D002086FE000899
:1097D000F0B58FB00D908848007880028749401816
:1097E0008749802200F040F9002804D0FFE70EA846
:1097F00001210170FCE082480C900C9800680D99E2
:1098000008610C9880880D9988820C98C0880D9901
:1098100008830C9800890D997C2288520C98408905
:109820000D997E2288520C9880890D999822885231
:109830000C98C0890D999A2288520C98008A0D992B
:109840008C2288520C98408A0D99A02288520C983C
:10985000808A0D99A82288520C9880690D998022DF
:1098600088500C98C0690D99842288500C98006A21
:109870000D99882288500C98406A0D999022885042
:109880000C98806A0D999C2288500C98C06A0D999A
:10989000A42288500C98006B0D99AC2288500C982B
:1098A000406B0D9988670C98806B0D9994228850B5
:1098B0000C98808F0D99522288520C98C08F0D9968
:1098C0005023C8520C98006C0D99C8650C9844211F
:1098D000405A0D9C542560530C984624005B0D9E05
:1098E0005627F0530C984826805B0B900D980A90F1
:1098F000582009900B9808910A990792099A885262
:109900000C984A21405A0D9A90860C984C22805A05
:1099100006900D980590069804910599C8860C98B4
:109920004E21405A03900D9802900398019102999C
:1099300008870C98C05A0D9948870C980799405A87
:109940000D9B98870C98405B0D9BD8870C98C05B4B
:109950000D9B402558530C98099BC05A0D9D4227DA
:10996000E8530C985A25405B0D9D089FE8530C98CE
:109970005C25405B0D9D28530C985E24005B0D9C7C
:10998000A0530C986024005B0D9C049D60530C98C0
:109990006224005B0D9CA0520C986422805A0D9AA0
:1099A000019C10530C98406F0D9A50600C986C22DB
:1099B000805A7C2804D0FFE70EA80121017017E02F
:1099C0000C986E21405A002804D0FFE70EA8012110
:1099D00001700DE00C987021405C2B2804D0FFE74B
:1099E0000EA80121017003E00EA800210170FFE71D
:1099F0000EA800780FB0F0BDE075FF1F00F8FF075C
:049A0000E80A002050
:109A040080B582B013480078800213494018694633
:109A1400012200F027F8002804D0FFE701A8012163
:109A2400017012E0684600782B2807D0FFE70C4845
:109A340005F07EFD01A901220A7006E0074805F041
:109A440077FD01A900220A70FFE701A8007802B09F
:109A540080BDC046E075FF1F70F8FF07F1DE000807
:049A6400DBDE00083D
:109A680087B002ABD86099605A6000201860D86847
:109A7800596840181549097889020122D2068918BF
:109A88008842009304D9FFE706A80121017019E074
:109A9800002000990860FFE7009801684268914239
:109AA8000CD2FFE70098C1680268895C8368995402
:109AB800FFE700980168491C0160EDE706A800214E
:109AC8000170FFE706A8007807B07047E075FF1F30
:109AD80010B588B00790794805F028FD78490691B7
:109AE80078490A68069B1A608A88069B9A80CA8801
:109AF800069BDA800A89069B1A814A89069B5A8145
:109B08008A89069B9A81CA89069BDA810A8A069BFA
:109B18001A824A8A069B5A828A8A069B9A828A698C
:109B2800069B9A61CA69069BDA610A6A069B1A62F1
:109B38004A6A069B5A628A6A069B9A62CA6A069BA6
:109B4800DA620A6B069B1A634A6B069B5A638A6B36
:109B5800069B9A638A8F069B9A87CA8F069BDA8729
:109B68000A6C069B1A6444228B5A069CA35246220E
:109B78008B5A069CA35248228B5A069CA3524A220F
:109B88008B5A069CA3524C228B5A069CA3524E22F7
:109B98008B5A069CA35250228B5A069CA3525222DF
:109BA8008B5A069CA35254228B5A069CA3525622C7
:109BB8008B5A069CA35258228B5A069CA3525A22AF
:109BC8008B5A069CA3525C228B5A069CA3525E2297
:109BD8008B5A069CA35260228B5A069CA35262227F
:109BE8008B5A069CA3526422895A069B995206995D
:109BF8008A6E521C8A6606996C227C238B520699BF
:109C08006E2200238B52069970222B238B540290CC
:109C1800FAF79EFC7D21C90001900846FAF79CFBE3
:109C280029490968C907002906D0FFE726480168BD
:109C3800012291430160FFE72448022101603F218E
:109C480041600121816005A9FAF7D2FE002802D0FF
:109C5800FFE7FFE7FEE71E48007880021D4940182D
:109C6800049000200390FFE70498194909788902B5
:109C7800194A8918884217D2FFE704990398C00047
:109C88000F4A131812585B680120FAF7E3FB002803
:109C980007D1FFE70498083004900398401C03900C
:109CA80001E0FFE7FEE7DFE7FAF790FC079900908D
:109CB8000846FFF789FD08B010BDC0460ADF000856
:109CC800E80A0020FCD9000814200240B80D002042
:0C9CD800E075FF1F00F8FF077CF8FF0795
:109CE40010B588B00790594805F022FC58490691F0
:109CF40058490A68069B1A608A88069B9A80CA8813
:109D0400069BDA808A8F069B9A870A6C069B1A64E4
:109D140044228B5A069CA352CA8F069BDA8746229A
:109D24008B5A069CA35248228B5A069CA3524A2261
:109D34008B5A069CA3524C228B5A069CA3524E2249
:109D44008B5A069CA35250228B5A069CA352522231
:109D54008B5A069CA35254228B5A069CA352562219
:109D64008B5A069CA35258228B5A069CA3525A2201
:109D74008B5A069CA3525C228B5A069CA3525E22E9
:109D84008B5A069CA35260228B5A069CA3526222D1
:109D94008B5A069CA3526422895A069B99520290BC
:109DA400FAF7D8FB7D21C90001900846FAF7D6FAE4
:109DB40029490968C907002906D0FFE72648016830
:109DC400012291430160FFE72448022101603F2101
:109DD40041600121816005A9FAF70CFE002802D038
:109DE400FFE7FFE7FEE71E48007880021D494018A0
:109DF400049000200390FFE7049819490978890228
:109E0400194A8918884217D2FFE704990398C000B9
:109E14000F4A131812585B680120FAF71DFB00283B
:109E240007D1FFE70498083004900398401C03907E
:109E340001E0FFE7FEE7DFE7FAF7CAFB07990090C6
:109E44000846FFF7C3FC08B010BDC04620DF000879
:109E5400E80A0020FCD9000814200240B80D0020B4
:0C9E6400E075FF1F00F8FF077CF8FF0707
:109E7000F0B593B00A46129011A80170A1490C9058
:109E800008460B9205F056FB9F49109112990969FB
:109E9000109A11601299898A109A91801299098BEF
:109EA000109AD18012997E22895A109A5181129962
:109EB0009822895A109A918112999A22895A109A55
:109EC000D18112998C22895A109A11821299A0225A
:109ED000895A109A51821299A822895A109A91820D
:109EE000129980228958109A916112998422895876
:109EF000109AD161129988228958109A1162129988
:109F000090228958109A516212999C228958109A6D
:109F100091621299A4228958109AD1621299AC22A6
:109F20008958109A11631299896F109A5163129986
:109F300094228958109A916312995222895A109B3F
:109F4000998712995023C95A109CE1871299C96DBB
:109F5000109C216412995424095B109D4426A95336
:109F600012995625495B109F0A9046203952129942
:109F70005827C95B099010980890482007900898C6
:109F80000692079A81521298808E10994A2288521E
:109F90001298C08E109905904C2004900598039259
:109FA000049A88521298008F10994E228852129863
:109FB000408F1099C8521298808F1099069BC852F2
:109FC0001298C08F1099085312984021405A109946
:109FD000485312984221405A1099C8531298805BF6
:109FE00010995A24085312980999405A109C5C25DC
:109FF00060531298079C005B109D5E26A853129830
:10A00000039D405B109E6027F0531298049E805B76
:10A01000109F622178521298805A109964228852B7
:10A020001098816E491C816610986C217C224252E6
:10A0300010986E2100224252109870212B22425417
:10A040000C980178002908D0FFE7304805F072FA33
:10A0500012994968109A5167FFE7FAF77DFA7D2156
:10A06000C90002900846FAF77BF929490968C9072F
:10A07000002906D0FFE726480168012291430160CC
:10A08000FFE72448022101603F21416001218160F6
:10A090000FA9FAF7B1FC002802D0FFE7FFE7FEE7BF
:10A0A0001D48007880021D4940180E9000200D9038
:10A0B000FFE70E98184909788902194A89188842D9
:10A0C00017D2FFE70E990D98C0000F4A13181258C7
:10A0D0005B680120FAF7C2F9002807D1FFE70E9864
:10A0E00008300E900D98401C0D9001E0FFE7FEE750
:10A0F000DFE7FAF76FFA129901900846FFF768FB5D
:10A1000013B0F0BD39DF0008E80A00204FDF000877
:10A1100014200240B80D0020E075FF1F00F8FF0773
:04A120007CF8FF07C1
:10A1240080B582B0019001980F494143080C00901A
:10A1340000980E490968401A009000980C49414360
:10A14400009100980B49096805F0DEFA0090009828
:10A1540009494018009000980A2105F0D5FA0749EA
:10A16400CC22885202B080BDE40C0000F80D00201F
:10A17400A0860100000E002030750000C0080020F9
:10A1840080B58AB009900891314801688A09891A12
:10A1940001600999026851180160006880090790FC
:10A1A4002C4801688A09891A0160089902685118C3
:10A1B400016000688009069007980699401A01F02A
:10A1C400D1FF059005982449CA228A5A0490104662
:10A1D400039101F0C7FF049902900846029901F027
:10A1E4006BFE01F0C1FC00221C4B019201F01AFC31
:10A1F40002F0F4F80590059801F0B6FC184A194BE2
:10A2040001F038FD184B019A04F099FB01F08EFF20
:10A21400D821039A50505058DC215158884206DD09
:10A22400FFE70D48D8214158DC228150FFE70A4856
:10A23400D8214158E0228058814206DAFFE70648D7
:10A24400D8214158E0228150FFE70AB080BDC046C2
:10A25400F00D0020F40D0020C00800200000F040A4
:0CA2640089E1CCEFA7CC8CBF000040408B
:10A2700070B59EB000201D901C901B901A901990F4
:10A2800018901790169015901490139012901190AA
:10A2900010907C48C16DE12212014A430F92E421E3
:10A2A000405800281CD4FFE776485221415A0E90AE
:10A2B000084601F0B9FC0022734B01F0B5FB159183
:10A2C0001490E4200E99085801F0AEFC149A159BE6
:10A2D00004F037FB01F02CFFF0210E9A505050E0B3
:10A2E0006848E42141580D90084601F09DFC1B91FF
:10A2F0001A901A981B990D9AD36D14240C90184635
:10A300000B91214605F020FA01F020FC0C9A0A90EE
:10A3100010460B9B099119460A9A099B01F084FB90
:10A320001D911C901D980121C90748401D90502087
:10A330000D99085A01F078FC0022534B089201F065
:10A3400073FB1991189018981999504B089A01F0BD
:10A3500093FC1D9A1C9B0790184606911146079A7C
:10A36000069B02F0DBFA179116901A981B99169A21
:10A37000179B04F0E6FA01F0DBFEF0210D9A505035
:10A38000FFE74048F0214158CA17F823C458054652
:10A39000F8356E6861185641C1506E60C0586968E2
:10A3A0000F9AD317101A8B4108DAFFE70F98C117DD
:10A3B000344AF823D050F8325160FFE73148C16D7C
:10A3C0005422825A4A4364210590104605F0BCF994
:10A3D000002111911090D8200599085858228A5AC6
:10A3E00090420FDDFFE72748E4214058C117119A3A
:10A3F000109BC01A914105DAFFE725480188491CE6
:10A40000018003E0224800210180FFE72048008806
:10A4100000B21C495622895A884208DDFFE70F988E
:10A42000C117184AF823D050F8325160FFE7154899
:10A43000F82141580246F832526804900846114605
:10A4400001F054FB0F9A03901046029101F0ECFBCF
:10A45000039A01901046029B00911946019A009BB5
:10A4600001F0E2FA13911290129813990022094B0D
:10A4700004F067FA01F05CFE01210902049A5050D1
:10A480001EB070BDC0080020000059400000F0BFA1
:08A49000280E0020006AF840CC
:10A4980080B586B0194805900598008801F074FECB
:10A4A800049004988B21C905029101F09DFE049047
:10A4B80004981349019101F0FDFC01F0CDFC11490C
:10A4C80008601148059005980088009101F05CFE2D
:10A4D80003900398029901F087FE0390039801996D
:10A4E80001F0E8FC01F0B8FC084908600868009928
:10A4F8000A68801A064A106006B080BDA875FF1F5A
:10A5080000803B45F80D0020CA75FF1FFC0D002098
:04A51800000E002011
:10A51C0080B586B00590134801688A09891A0160D4
:10A52C00059902685118016000688009049004982C
:10A53C000D4941430D4803900846039905F0FEF878
:10A54C000B49C8228852C83104980A4A0290104616
:10A55C00029A0191114605F0F1F80199488006B074
:10A56C0080BDC046040E0020E40C0000FFFF00007C
:08A57C00C00800203CF6C309F1
:10A5840080B584B003900E4801688A09891A016075
:10A5940003990268511801600068800902900298CA
:10A5A4000849CA228A5A42431F205043064A01914D
:10A5B400114605F0C7F8D421019A505004B080BD6B
:0CA5C400080E0020C0080020FFFF00006F
:10A5D00080B582B00190019819494143C817000C19
:10A5E0000818001400900098164940180090009830
:10A5F00064214143009100980A2105F087F812492F
:10A60000CE228852885ED022895E884206DDFFE72E
:10A610000D48CE21415AD02281520EE00A48CE2167
:10A62000415ED222805E814206DAFFE70648CE21F3
:10A63000415AD2228152FFE7FFE702B080BDC046F7
:0CA64000E40C0000A8FDFFFFC008002093
:10A64C0080B58AB0099008910792089804900998EF
:10A65C00182141432548401818300390039840694D
:10A66C000028029008D0FFE70298012819D0FFE7D4
:10A67C00029802282CD032E0039804F04FF8059091
:10A68C0005980799884203D2FFE70020069007E05F
:10A69C000798069003980499079A04F097FEFFE731
:10A6AC0020E0039804F03AF8059005980799884241
:10A6BC0003D2FFE70598019002E007980190FFE7AD
:10A6CC000198069003980499069A04F07FFE09E01D
:10A6DC0003980499079A04F0B9FE069002E0002052
:10A6EC000690FFE706980AB080BDC046680B0020B4
:10A6FC0080B588B0884841218900405E002808D088
:10A70C00FFE7854841218900405E401C002800D0AD
:10A71C00ADE08148D8214158008F814213DDFFE71D
:10A72C00834804F001FF7C494122920001238B52A3
:10A73C00052109071A0200230790084611461A46FC
:10A74C0003F003FD92E07448E42141583E22805E00
:10A75C007D22D2004243914214DDFFE7734804F09E
:10A76C00E3FE6D494122920002238B520521090719
:10A77C000122120200230690084611461A4603F0E5
:10A78C00E4FC72E06448CE21415E4022805E81424E
:10A79C0014DDFFE7644804F0C7FE5F4941229200D4
:10A7AC0003238B5205210907012212020023059075
:10A7BC00084611461A4603F0C8FC55E05648CC2111
:10A7CC00415E4022805E814214DDFFE7554804F073
:10A7DC00ABFE51494122920004238B5205210907FB
:10A7EC000122120200230490084611461A4603F077
:10A7FC00ACFC38E04848CE21415E4422805E814268
:10A80C0013DAFFE7464804F08FFE434941229200D9
:10A81C0005238B52190701221202002303900846CC
:10A82C0011461A4603F091FC1CE03B48CC21415EDA
:10A83C004422805E814214DAFFE7384804F074FE4B
:10A84C0035494122920006238B520521090701222A
:10A85C00120200230290084611461A4603F075FCBA
:10A86C00FFE7FFE7FFE7FFE7FFE7FFE7FFE72A4820
:10A87C0041218900405E00284CD0FFE72648D821B2
:10A88C004158408F814245DAFFE72348E421415883
:10A89C003E22805E7D22D200424391423ADAFFE7AB
:10A8AC001D48CE21415E4222805E814232DAFFE7B2
:10A8BC001948CC21415E4222805E81422ADAFFE7B0
:10A8CC001548CE21415E4622805E814222DDFFE7A3
:10A8DC001148CC21415E4622805E81421ADDFFE7A1
:10A8EC000D4841218900405E022812D0FFE7114833
:10A8FC0004F01AFE08494122920000238B520521D4
:10A90C0009070122130201900846194603F01DFCA9
:10A91C00FFE7FFE708B080BDC0080020E9FB000896
:10A92C00C5FB0008A3FB000880FB000867FB0008C0
:08A93C0046FB00080BFC0008BB
:10A9440080B582B01B4801900198022101610198F1
:10A9540041610198184981610198184AC2610198BE
:10A9640001229202026201980022826201984262EC
:10A974000198C2620198816401981149C1640198E7
:10A984001021016501988265019842650198C265AC
:10A994000198C01D0B4904F063FF01990A4A009015
:10A9A4000846114604F05CFF019920228A7102B026
:10A9B40080BDC046680B00203FFF00088C000020CB
:0CA9C400A80D002048FF00084CFF000810
:10A9D00080B586B0059004910392FFE70D4800789A
:10A9E000002803D1FFE7FFF7ADFFFFE7FFE7EFF335
:10A9F0001080012181F31088019005980499039A31
:10AA0000FFF724FE0290019880F31088029806B0A8
:08AA100080BDC046680B002068
:10AA180080B588B0884883214900405E002808D066
:10AA2800FFE7854883214900405E401C002800D08C
:10AA3800ADE08148D8214158808E814213DAFFE782
:10AA4800824804F073FD7C498322520001238B5213
:10AA5800052109075A0200230790084611461A469D
:10AA680003F075FB92E07448E42141583C22805E73
:10AA78007D22D2004243914214DAFFE7724804F083
:10AA880055FD6D498322520002238B520521090787
:10AA98000122520200230690084611461A4603F086
:10AAA80056FB72E06448CE21415E4822805E8142B6
:10AAB80014DDFFE7634804F039FD5F498322520043
:10AAC80003238B5205210907012252020023059016
:10AAD800084611461A4603F03AFB55E05648CC2181
:10AAE800415E4822805E814214DDFFE7534804F04E
:10AAF8001DFD51498322520004238B520521090769
:10AB08000122520200230490084611461A4603F017
:10AB18001EFB38E04848CE21415E4C22805E8142CF
:10AB280013DAFFE7464804F001FD43498322520047
:10AB380005238B521907012252020023039008466D
:10AB480011461A4603F003FB1CE03B48CC21415E4A
:10AB58004C22805E814214DAFFE7384804F0E6FCB4
:10AB680035498322520006238B5205210907012209
:10AB7800520200230290084611461A4603F0E7FAEB
:10AB8800FFE7FFE7FFE7FFE7FFE7FFE7FFE72A4801
:10AB980083214900405E00284CD0FFE72648D82191
:10ABA8004158C08E814245DDFFE72348E4214158E2
:10ABB8003C22805E7D22D200424391423ADDFFE78B
:10ABC8001D48CE21415E4A22805E814232DAFFE78B
:10ABD8001948CC21415E4A22805E81422ADAFFE789
:10ABE8001548CE21415E4E22805E814222DDFFE77C
:10ABF8001148CC21415E4E22805E81421ADDFFE77A
:10AC08000D4883214900405E022812D0FFE7104812
:10AC180004F08CFC08498322520000238B52052142
:10AC280009070122530201900846194603F08FFADA
:10AC3800FFE7FFE708B080BDC0080020F1FA000870
:10AC480013FB0008CEFA0008B5FA000893FA0008CA
:04AC580037FB0008BE
:10AC5C00044883214900044A42524121890042524E
:0CAC6C007047C046C0080020FFFF000039
:10AC780010B586B0089C0490039102920193049841
:10AC8800002804D1FFE705A8012101706FE00498AE
:10AC980080214058002808D1FFE704987C21002231
:10ACA80042540498FEF708F8FFE70498802124220C
:10ACB8004250049800680168012291430160049899
:10ACC800FBF7D4FF012804D1FFE705A80121017093
:10ACD8004DE00498806A002804D0FFE7049803F048
:10ACE80004FCFFE704980068816801229303194374
:10ACF8008160049800688068D103884303990843F9
:10AD08000499096888600298400500900198000439
:10AD180000990143009104980068006816490840AA
:10AD28000099084304990968086004980068416814
:10AD3800D3051943416004980068016893061943D4
:10AD48000160049800684069FF21090608400899D5
:10AD58000843049909684861049800680168114328
:10AD680001600498FCF7CCFF05A90870FFE705A867
:0CAD7800007806B010BDC046FFFF00FCD4
:10AD8400B0B588B00D9C0C9D079006910592049374
:10AD9400069807990860079800684C49016007986D
:10ADA40000684B21090241600798006801210A03E9
:10ADB4008260079800680022C260079800688902D0
:10ADC4000161079800680C2141610798006882615D
:10ADD40007980068C26107980068026207980068D3
:10ADE400426207980068826205980799096848607A
:10ADF400049800280AD1FFE70798006801218A0215
:10AE04000261079800680903816017E0049801282B
:10AE14000BD1FFE7079800680321490201610798F5
:10AE2400006801210903816007E007980068002198
:10AE34000161079800688160FFE7FFE70C9801282B
:10AE440005D1FFE7079800680021C16005E0079875
:10AE5400006801214903C160FFE7079800680D9964
:10AE64000390084600F070FE0022194B029203F092
:10AE740066FD01F043F9009003980299029A029B3F
:10AE8400FFF7F8FE002803D0FFE703F047FCFFE7D5
:10AE94000798006803F005FC002803D0FFE703F0DF
:10AEA4003DFCFFE707980168273001221202019058
:10AEB40008460199FCF70EFE002805D0FFE7054877
:10AEC40004F036FBFFE7FEE708B0B0BD00380140F0
:08AED40000000C40AFFE000875
:10AEDC0010B58AB01C4608900791069205A803701D
:10AEEC0000783B49098B88420DD0FFE705A8007814
:10AEFC00002808D0FFE70898069B06210B2203F0D8
:10AF0C006CFC099060E0079881780902C0780818F9
:10AF1C000490079801790902407908180290029868
:10AF2C00002804D0FFE702987E2809D3FFE7089891
:10AF3C00069B03210191019A03F04FFC099043E019
:10AF4C00049802994018401E8C2808D3FFE70898F3
:10AF5C00069B0321022203F040FC099034E0089880
:10AF6C000699032242540698401C06900298400011
:10AF7C000899069A88540698401C069004980390E9
:10AF8C00FFE703980499029A8918884219D2FFE7BF
:10AF9C00039840000E4908184078089A069BD05434
:10AFAC000698401C069003984000085C0899069A85
:10AFBC0088540698401C0690FFE70398401C0390A9
:10AFCC00DFE706980990FFE709980AB010BDC04664
:04AFDC00C008002089
:10AFE00080B586B0049004982730029004984521DB
:10AFF000C9004058039002980078019003980428F3
:10B0000006D8FFE7049803F0E3FB0020059024E056
:10B010000298039903F000FC401C002806D1FFE7CA
:10B02000049803F0D5FB0020059016E00198002855
:10B0300003D1FFE7022005900FE001980849098B32
:10B04000884203D1FFE70220059006E0FFE704985D
:10B0500003F0BEFB00200590FFE7059806B080BD19
:04B06000C008002004
:10B0640080B586B0049003910292019301982D4912
:10B07400098B88420CD0FFE70198002808D0FFE72D
:10B084000498029B06210B2203F0ABFB059046E0DB
:10B09400039881780902C0780818009000988C28D9
:10B0A40008D3FFE70498029B0621022203F099FBD0
:10B0B400059034E00398007900994900194A511821
:10B0C40048700398407900994900505404980299B3
:10B0D400062242540298401C02900098000A0499E7
:10B0E400029A88540298401C029000980499029A8B
:10B0F40088540298401C0290039800790499029A9B
:10B1040088540298401C0290039840790499029A4A
:10B1140088540298401C029002980590FFE7059815
:08B1240006B080BDC008002048
:10B12C0085B00490039102A81C4901800020019075
:10B13C00FFE70198039988422CD2FFE70498019904
:10B14C00405C0299414002A8018008200090FFE772
:10B15C000098002819D0FFE702A80088C007002833
:10B16C0009D0FFE702A801884908018002990C4A1E
:10B17C005140018004E002A8018849080180FFE7E2
:10B18C00FFE70098401E0090E2E7FFE70198401CA3
:10B19C000190CEE702A8008805B07047FFFF0000C1
:04B1AC0001A00000FE
:10B1B00080B58AB008900791069205930598454995
:10B1C000098B88420CD0FFE70598002808D0FFE7DC
:10B1D0000898069B06210B2203F005FB099075E0F9
:10B1E000079881780902C0780818049007980179B7
:10B1F000090240790818039007200190039800285D
:10B2000004D0FFE703987C2808D3FFE70898069B43
:10B210001021032203F0E7FA099057E004980399FC
:10B220004018401E8C2808D3FFE70898069B102181
:10B23000022203F0D8FA099048E004980290FFE750
:10B2400002980499039A8918884217D2FFE7079851
:10B250000199405C029949001E4A511848700798AC
:10B260000199081840780299490050540198801CAF
:10B270000190FFE70298401C0290E1E708980699C8
:10B28000102242540698401C06900498000A08991F
:10B29000069A88540698401C069004980899069AC5
:10B2A00088540698401C06900398000A0899069A4C
:10B2B00088540698401C069003980899069A88546A
:10B2C0000698401C069006980990FFE709980AB076
:08B2D00080BDC046C00800204B
:10B2D80010B58AB0099009980068C0690890099863
:10B2E8000068006807900998006840680690099807
:10B2F80000688068059008980F2108400490049819
:10B3080000286CD0FFE70598A549084207D1FFE758
:10B3180007A8008809214901084260D0FFE708A86A
:10B328000078C007002810D0FFE707A84078C007BA
:10B3380000280AD0FFE709980068012101620998EE
:10B34800882283580B438350FFE708A800788007BA
:10B35800002811D5FFE705A80078C00700280BD002
:10B36800FFE709980068022101620998882142587C
:10B3780004231A434250FFE708A800784007002832
:10B3880011D5FFE705A80078C00700280BD0FFE714
:10B39800099800680421016209988821425802230B
:10B3A8001A434250FFE708A800780007002815D57F
:10B3B800FFE707A800788006002805D4FFE705986E
:10B3C800774908420AD0FFE7099800680821016216
:10B3D8000998882283580B438350FFE7FFE708A8A2
:10B3E8004078000700281DD5FFE707A8C078400768
:10B3F800002806D4FFE705A880780006002811D5A4
:10B40800FFE7099800680121CA02026209988422AC
:10B418002023835009988022835062480175624A2C
:10B428008154FFE708A800788006002832D5FFE796
:10B4380007A800788006002806D4FFE705A8C0788A
:10B44800C006002826D5FFE70998842140582228FD
:10B4580018D1FFE753484521C9004058FF2811D8A3
:10B46800FFE709980068406A4E494522D2008B5888
:10B47800CB18272418558858401C88504A48012260
:10B488000A5406E00998006881690822114381611D
:10B49800FFE7FFE708A800780006002818D5FFE7AF
:10B4A80007A800780006002806D4FFE705A88078DA
:10B4B800000600280CD5FFE73A48016802900846C4
:10B4C80004F060F8232000010121029A1154FFE7DB
:10B4D80008A800784006002812D5FFE707A80078DA
:10B4E800400600280CD5FFE72E48262100224254AA
:10B4F800099803F034F90998842122224250FFE781
:10B50800099888214058002848D0FFE709988421E5
:10B518002222425008A800788006002817D5FFE7A5
:10B5280007A800788006002806D4FFE705A8C07899
:10B53800C00600280BD5FFE7099800688169082232
:10B5480011438161099888210022425025E008A80A
:10B558000078000600281FD5FFE707A80078000636
:10B56800002806D4FFE705A880780006002813D530
:10B57800FFE70C4826210022425409990190084609
:10B5880003F0EDF80998842122224250232000017B
:10B598000121019A1154FFE7FFE7FFE70AB010BD48
:0CB5A800010000108C04002031020000A3
:10B5B40080B588B000200590019000F009FA802041
:10B5C40003901F4800687F2109020840000A049084
:10B5D40001980590FFE705980399884224D2FFE774
:10B5E400174801687F2212029143059A12021143FF
:10B5F400016002200790FFE70798022804D1FFE7C3
:10B6040000F072F90790F7E7002006900798069972
:10B61400081806900698059989000A4A5050FFE7D1
:10B624000598401C0590D6E7054801687F22120260
:10B634009143049A12021143016008B080BDC046D0
:08B6440004100240C0060020C2
:10B64C0080B58AB0FFE725480168012252041143F6
:10B65C0001600068104005900598FFE720482149DB
:10B66C0001600490FAF748FF1F49049AD160002149
:10B67C005160116191600390104603F057FB002854
:10B68C0002D0FFE7FFE7FEE70020069001210791BB
:10B69C000C2108910990124906AA029008461146FD
:10B6AC00029A03F0C3FC002802D0FFE7FFE7FEE795
:10B6BC000B480221002203F067FC002802D0FFE7B0
:10B6CC00FFE7FEE71520002101900091009A02F09F
:10B6DC00A6FC019803F008FB0AB080BD40100240A4
:0CB6EC00040D002000440140FFFF00009E
:10B6F80080B586B005900598007F012875D1FFE7D1
:10B708003B48006801280AD1FFE70598002102F0AC
:10B71800A7FB3A49086036480221016064E03448D2
:10B72800006802285FD1FFE705980021049102F024
:10B7380097FB304908601520039103F0D7FA2E488B
:10B748000499FAF70FFF059909680222D2430A61A2
:10B7580003990A68294B1B689A421AD9FFE72548BA
:10B76800006826490968401A2649086008680003E5
:10B77800254988420CD8FFE7244803F0D7FE214921
:10B7880009680903224A0290104603F0CFFEFFE73A
:10B7980025E0184800681949096888421CD2FFE763
:10B7A8001648006813490968081A154940181549C8
:10B7B800086008680003144988420CD8FFE713485A
:10B7C80003F0B4FE0F4909680903114A01901046B5
:10B7D80003F0ACFEFFE701E0FFE7FEE7FFE7044800
:10B7E80003210160FFE7FFE7FFE706B080BDC04621
:10B7F8000C0E0020100E0020040D0020180E002052
:10B80800FFFF00001C0E00203F5DC600E9FE000897
:04B81800FAFE00082C
:10B81C0080B586B0002002900590FFE705987F2840
:10B82C0038D8FFE7059880002B4908580190002074
:10B83C0003900490FFE704987F2811D8FFE7019844
:10B84C0004998900244A5158884204DDFFE7039883
:10B85C00401C0390FFE7FFE70498401C0490EAE7C4
:10B86C00059803991B4A50540398105C00280CD17E
:10B87C00FFE70298012805D1FFE7184803F054FEB2
:10B88C00FFE7FEE701200290FFE7FFE70598401C69
:10B89C000590C3E70E484021017000200590FFE79A
:10B8AC0005987F2811D8FFE7094800780599094ABF
:10B8BC00515C884204D1FFE7059805490870FFE701
:10B8CC00FFE70598401C0590EAE706B080BDC0462E
:10B8DC002B0E0020640A0020C00600201AFC000871
:10B8EC0010B586B03348006804280FD1FFE7314803
:10B8FC000121016030480021FAF7AAFD15210390BF
:10B90C00084603F0FDF9022005904FE02948006835
:10B91C00032803D0FFE70220059047E02548006884
:10B92C0003283ED1FFE7152003F0DEF92248002161
:10B93C00FAF716FE1F4904220A60204909680029FB
:10B94C0008D0FFE71E48006800031E490A6810185B
:10B95C000860FFE719480068092807D8FFE717486F
:10B96C000168491C0160022005901FE00020049032
:10B97C001249086010490968896A491C114A136800
:10B98C000A240290184601912146009203F0D6FE3B
:10B99C00019948430490029800990860049A059212
:10B9AC0004E0FFE7FFE700200590FFE7059806B0ED
:10B9BC0010BDC0460C0E0020040D0020140E0020FB
:08B9CC001C0E0020200E0020DB
:10B9D40080B5FFF739FE02480421016080BDC046EE
:04B9E4000C0E002025
:10B9E80030B401256D054C00E54215D85C00E542F0
:10B9F80012D80C001C436400044314430CD005D235
:10BA080082428B418041404230BC7047904299410C
:10BA18008041404230BC7047002030BC7047C0466F
:10BA2800F0B40125ED070C005C402C40A446AE0A9A
:10BA38004C18DF18F4423DD2F74245D2640D4CD081
:10BA48007F0D3CD0E41BC9022943CF0ADB022B43FC
:10BA5800DB0A0600B61A9F4104D2013CB6197F41A1
:10BA6800B6185F416812800D241838DD001884422A
:10BA780025D8E80C0021B6197F41B61A9F4103D397
:10BA880040414941F7D304E0B6185F4100184941E5
:10BA9800F1D32405B6197F41B61A9F4105D3374320
:10BAA800C20717430022012F5041614162461143EA
:10BAB800F0BC70470CD100420AD1F74208D20020EE
:10BAC800C143490D0905F1E7124201D1F74206D0F9
:10BAD8000020C143090DC904EAE77F0DF8D0002012
:04BAE8006146E5E7E7
:10BAEC000B0003432BD0CA0FD200043212023D329A
:10BAFC00094203D5002349424042994102D1010039
:10BB0C000020203A01231B04994204D2103A090464
:10BB1C00030C19430004094203D4013A00184941AB
:10BB2C00FBD58446C00A4B051843C90A1205634667
:10BB3C005B055B4102D3012B0023584151417047F7
:10BB4C0042221201033A0146004207D002D4013AC4
:10BB5C000018FCD51205C30A400599187047C04659
:10BB6C0041008C46012212068A420BD8090938235F
:10BB7C001B06C918C30FDB07194340076346DA429B
:10BB8C0004D27047C10FC9070020704703D1382376
:10BB9C001B06C918704738231B06C9180122D2048A
:04BBAC00114370478A
:10BBB000012212064300DA4211D84B00DA420ED8B5
:10BBC00002000A43520008D003D281428041013072
:10BBD0007047884280410130704701207047002043
:04BBE0007047C046A4
:10BBE40030B401256D054C00E54215D85C00E542F2
:10BBF40012D80C001C436400044314430FD005D234
:10BC040082428B418041013030BC7047904299415F
:10BC14008041013030BC7047002030BC70470120A7
:04BC240030BC704779
:10BC2800004201D4054A1047404200B5FFF78AFF99
:10BC380008BC0122D2071143184700004DBB000879
:10BC4800012212064300DA420FD84B00DA420CD820
:10BC580002000A43520008D003D288428041404281
:10BC68007047814280414042704700207047C0467B
:10BC7800F0B40125ED070F005F405AD48B4200D184
:10BC8800824205D950404240504059404B405940AB
:10BC98004E18760DDF187F0D3BD0741C640529D033
:10BCA800F41B352C26D80E0DDB022B43DB0AC90208
:10BCB8002943C9121700202C1ED2E741E240574001
:10BCC800E3415A40A340E3405A40002480185941B8
:10BCD8000AD3B21C520521D0C207012F62411700B6
:10BCE8004008CB0718434908013636054208AF41DA
:10BCF80060417141F0BC7047203C06D01F00E7410D
:10BD0800E3405F400024012A6741C0186141EBD33A
:10BD1800DFE7002EEED129400020EBE701363105A0
:10BD28000020E7E7E742E5D10020C143090DC90437
:10BD3800E0E76B400E00871A9E4104D26E40C01B9C
:10BD4800B141D21973414E18DF18AC0AE642E9D264
:10BD5800760D7F0D31D0F41B362CCBD8B4460E0DA2
:10BD6800DB022B43DB0AC9022943C90A012C32D85A
:10BD780004D1D4075208DF073A435B08EF0A64424C
:10BD8800904199411ED0002239424DD12419404199
:10BD980049410124394204D101340018494139424A
:10BDA800FAD06246A24204D9361B013E36058919EB
:10BDB800A0E7F10AC90700209CE736429AD1002083
:10BDC800002197E70200224394D0B842DED2010056
:10BDD80020002024E3D1202C13DD203CE241170071
:10BDE800A240E2405740E3415A40A340E3405A4052
:10BDF800012FBF410137174300227C4298419141EE
:10BE08000CE01700E741E2405740E3415A40A340A5
:10BE1800E3405A407C429041994100220F0303D2EB
:10BE2800013E241940414941013E36054708AC41CD
:08BE380050417141F0BC70475C
:10BE400002000A43520008D0884204D14000012178
:10BE50000906C84201D90020704701207047C0463A
:10BE600041000ED2090E7F390BD449421F3105D44F
:10BE700000020122D2071043C8407047012040420F
:08BE8000704700207047C04626
:10BE8800012212064300DA4211D84B00DA420ED8DA
:10BE980002000A43520008D003D288428041013090
:10BEA800704781428041013070470120704700206F
:04BEB8007047C046C9
:10BEBC0030B405004D400124E407254042004B00FE
:10BECC00120E32D01B0E3CD0FF2A33D0FF2B3FD0AA
:10BEDC00D21800022043000A09022143090AC4B205
:10BEEC004C43000AC3B24B43000A4843210A5B1877
:10BEFC00190A091801D44900013A080A7F3A2ADBC9
:10BF0C00FE2A0FD2D2051C43240601D00124214362
:10BF1C00C9B280295041802901D1400840002843F2
:10BF2C0030BC7047FF20C005F9E71B0EFF2B0AD071
:10BF3C002800F5E7400206D1FF2BF3D1490202D1CC
:10BF4C00F0E7FF2AF4D17F2000010C300005E7E771
:10BF5C004902F8D1E6E743020132E9D15B12023320
:08BF6C00E6D9D805E4E7C04660
:10BF74000122D20703004B403DD430B4431A01D20E
:10BF8400C01AC9184B004400240EFF2C29D02442A7
:10BF940024D01B0E20D0E31A182B1DDC09021143F8
:10BFA400C40D000210435D4219350A00AA40D209AB
:10BFB400D940451801D36D080234013CE405280A30
:10BFC4000121C9072D062A438A4160414100090E17
:10BFD400FF2901D3C00DC00530BC7047C00FC00796
:10BFE400FAE742001823DA41FF2AF5D07F20000146
:10BFF4000C300005F0E7A4465140431A02D25340E6
:10C00400C01AC9184B00090211431B0E4400240E28
:10C01400FF2C3DD01B4244D05B421B19012B0CD397
:10C024001ED1C30D4002401A0CD3DB050100400AA7
:10C03400C9059141584164467047C30D4002490007
:10C04400401AF8D0002101314000FCD38C4204D9BD
:10C054005B1ADB05400AC018EDE7180AC007EAE7D7
:10C06400192BE8D801330C00D940DC414C40012C99
:10C074004941C30D00021043441A01D4A4006408CA
:10C08400013BDB05200A240694415841644670476D
:10C09400FF2B01D04102CED07F2000010C300005DF
:0CC0A400C9E72442C7D10020C5E7C04610
:10C0B0000122D2075140014B1847000079BF000808
:10C0C00030B401256D054C00E54215D85C00E54211
:10C0D00012D80C001C436400044314430CD005D256
:10C0E000904299418041404230BC704782428B412E
:10C0F0008041404230BC7047002030BC7047C04691
:10C100004A1810D2520D40231B01D21A01320AD410
:10C1100052421F3209D4400DC90208430123DB07F4
:10C120001843D04070470020704700200138704706
:10C13000F4464A1805D2FFF7E5FF01D5C0174008BD
:10C14000604701235B05D34206D2FFF7DBFF01D531
:10C150000120C0074042604701D10042F5D00020D5
:08C16000013840087047C04699
:10C16800C20F12029D3201000CD001D5494202D4FF
:10C17800013A4900FCD5D205080A0906494100D30D
:08C18800012950417047C04637
:10C190009D2201000AD002D4013A4900FCD5D20503
:10C1A000080A0906494100D3012950417047C04699
:10C1B000012212064300DA420FD84B00DA420CD8B3
:10C1C00002000A43520008D003D28142804140421B
:10C1D0007047884280414042704700207047C04607
:10C1E000F0B40125ED076B40004C20477FBC0008F0
:10C1F00030B405004D400124E407254042004B00C7
:10C20000120E26D01B0E34D0FF2A2DD0FF2B35D096
:10C21000D21A000220430902214343084908A00D15
:10C220005B1A02D2013A5B005B185B008B4200D3C1
:10C230005B1A4041F9D37F3222DDFF2A06D2D205B4
:10C24000C91A8B425041284330BC7047FF20C005BB
:10C25000F9E71B0E03D0FF2B12D1490210D07F202B
:10C2600000010C300005EFE74002F8D1FF2BEDD1C3
:10C27000F5E7FF2AEAD14002F1D1E7E74902EED122
:04C280002800E1E7CA
:10C2840070B4012676054C005D00E6420CD8EE42FF
:10C294000AD825430543154303D0994204D190425B
:10C2A40002D1012070BC7047002070BC7047C046AA
:10C2B40030B401256D054C00E54215D85C00E5421B
:10C2C40012D80C001C436400044314430FD005D25D
:10C2D400904299418041013030BC704782428B4189
:10C2E4008041013030BC7047002030BC70470120D1
:04C2F40030BC7047A3
:08C2F800C00FC0077047C046EB
:08C30000490049087047C046DE
:10C308004200120E0AD0FF290BD07E3A0A60FF22A3
:10C31800D20590437E22D205104370470A60C00FB1
:04C32800C007704793
:10C32C004200120E06D0521804DDFF2A05D2C905B0
:10C33C0040187047C00FC0077047C00F0002FF3095
:04C34C00C005704771
:10C35000012849410020C043400501308842804106
:04C3600040427047A0
:10C3640042001FD0120EFF2A1DD07F3A12DB172A7B
:10C3740018DA0123DB05013BD340004208D5010054
:10C38400194005D098430121C905D1404018704790
:10C3940098437047004204D5BF2000028030000457
:10C3A4007047002070474102FCD07F2000010C3010
:04C3B40000057047C9
:08C3B800400040087047C04638
:10C3C000400000BAFF2801D00020704701207047CC
:10C3D00041000020FF221206013291424041704785
:10C3E0004B1801225205DA4217D25B0D0722D20107
:10C3F0009B1A0FD9FF2B13D2DB05CA0FD2071343A9
:10C400000903020D1143490AC200524100D901310A
:10C41000C8187047C80FC007704706D1004204D142
:10C42000C80F0002FF30C00570470123DB070A0078
:10C43000C900400F084398431A4010435B0A184351
:04C440007047C0463B
:10C44400F0B5C6460023904600B5002206000F0052
:10C45400FFF716FF002807D00023424630003900BA
:10C46400136004BC9046F0BD064A7B0094464246E5
:10C474005B0D63441360044B044A3B401A43300091
:10C484001100EEE702FCFFFFFFFF0F800000E03F1A
:10C49400F0B5C64600B5904682B0002200230F00D6
:10C4A4000400FFF7EDFE002816D17B005B0D104A57
:10C4B4004344934213DC4246002A01DB002B0EDB8B
:10C4C400002B09DD0B4A1B053A401A4320001100DA
:10C4D40002B004BC9046F0BD00200021F8E700F053
:10C4E400A9FB054B05491B68036001930020EFE796
:10C4F400FE070000FFFF0F8084DA00080000F07FD1
:10C50400F0B5C64600B582B004000D00FFF71EFF6B
:10C51400002800D097E020002900534A534BFFF72E
:10C5240061FA002800D094E020002900504A514BC1
:10C53400FFF7C4FD002805D00020002102B004BC90
:10C544009046F0BD20002900FFF7D8FE4A4A4B4B25
:10C55400FFF7B4FD002879D1002200232000290030
:10C56400FFF7A6FE002600287CD0454F20002900B6
:10C57400444A454B02F0E3F932003B00FFF77AFBF3
:10C58400FFF7D4FD8046FFF74DFB00223F4B06002A
:10C594000F0002F0D4F902000B0020002900FFF77D
:10C5A4001DFE3B4A04000D0030003900394B02F0F7
:10C5B400C6F902000B0020002900FFF75BFB020014
:10C5C4000B0006000F0002F0BAF904000D00324A15
:10C5D400324B02F0B4F9324A324BFFF74BFB2200E4
:10C5E4002B0002F0ACF900222F4BFFF743FB320083
:10C5F4003B0002F0A4F906000F00200029002B4A9A
:10C604002B4B02F09CF92B4A2B4BFFF733FB2200F8
:10C614002B0002F094F90022194BFFF72BFB320098
:10C624003B00FFF7DBFD444602000B0030003900FD
:10C63400FFF7F8F901340022114BFFF71BFB22002E
:10C64400FFF726FF7AE72000290077E700201B493F
:10C6540074E700F0EFFA1A4B1A491B680360019360
:10C6640000206BE7184F81E7EF39FAFE422E86402F
:10C67400D2BC7ADD2B2386C02342920CA19CC73BFB
:10C684000000E03F3CF92F9E2C15F73F0030E63FB9
:10C69400A80C615C10D02B3F1CDC586FA452F13EF7
:10C6A400E0F6B36FE4707C3F0000D03F0938DE6FE2
:10C6B400993F403FB35142718E71AC3F0000F03F4F
:0CC6C40084DA00080000F07F0000E0BFF6
:10C6D000F0B587B004000D00FFF73AFE002800D047
:10C6E000ACE00022002320002900FFF7CBFD00284A
:10C6F00000D0A7E00022002320002900FFF7E0FC83
:10C70000002800D09AE02000290005AAFFF79AFE31
:10C710005B4A5C4B04000D00FFF766F9002800D06F
:10C7200093E0059B0022013B200029000593564B16
:10C73000FFF756FD0122524204000D00FFF7AAFE4A
:10C740000022514BFFF798FA02000B00200029004D
:10C75000FFF76AF906000F0032003B003000390095
:10C7600002F0EFF8494A4A4B04000D0002F0E9F8E4
:10C77000484A494BFFF780FA484A00900191484BDC
:10C7800020002900FFF72CFD22002B0002F0D9F831
:10C79000444A454BFFF770FA009A019B02900391BF
:10C7A0002000290002F0CDF8404A414BFFF718FD68
:10C7B000029A039B009001912000290002F0C1F829
:10C7C0003C4A3D4BFFF70CFD02000B00009801991D
:10C7D000FFF72AF902000B002000290002F0B1F84F
:10C7E00032003B0002F0ADF8009001910598FFF790
:10C7F0001BFA009A019B04000D0030003900FFF77E
:10C800003BFA2E4A06000F00200029002C4B02F0B4
:10C8100098F802000B0030003900FFF72DFA0022D3
:10C8200006000F0020002900264B02F08AF80200C3
:10C830000B0030003900FFF71FFA01E00020224909
:10C8400007B0F0BD00202149FAE7214B002220006B
:10C850002900FFF7C5FC012206000F00524220000C
:10C860002900FFF717FE0022074BFFF705FA020029
:10C870000B0030003900FFF7D7F806000F006BE718
:10C88000CD3B7F669EA0E63F0000E03F29BD56B34A
:10C890001544E9BFEDAF16204A6230400FCE674B1A
:10C8A00080D541407E2615FA838073409AB5B31235
:10C8B000FF07504077900D9CFE0B8840A80C615CF0
:10C8C00010D02BBF0030E63F0000F87F0000F0FFE3
:04C8D0000000F03F35
:10C8D40070B500240E00211C051CFFF7AFFA0028D8
:10C8E4000FD16B001B0E7F3B0ED4162B0FDC094AB5
:10C8F400281CDA402B00934319003360FFF7D6FB62
:10C9040070BD3460201CFBE73460281CF8E73560F8
:08C91400201CF5E7FFFF7F0086
:10C91C00F0B54746CE46160080B51F0004000D004A
:10C92C0083B0002230003900414BFFF7A5FC0028F2
:10C93C003ED10022002320002900FFF79DFC002897
:10C94C0010D00022002330003900FFF745F90028F1
:10C95C0031D1002600273000390003B00CBC9046C2
:10C96C009946F0BD39003000FFF7DCFB8046FFF73D
:10C97C0055F932003B00FFF77FFC002824D1002240
:10C98C00002320002900FFF795FB002813D120007D
:10C99C002900FFF7AFFCFFF795FE02000B003000FB
:10C9AC00390001F0C8FFFFF7A7FD06000F00D2E722
:10C9BC0026002F00CFE700F039F91E4B00261B682C
:10C9CC001D4F01930360C6E74346002B21DB2CD09F
:10C9DC000123994642464B460026154F134207D079
:10C9EC003000390022002B0001F0A5FF06000F00DB
:10C9FC0043465B109846AED022002B002000290045
:10CA0C0001F099FF4B46424604000D001342EFD053
:10CA1C00E6E72B00220000200549FEF7FFFF434606
:10CA2C005B4204000D009846D2E70026004F92E7C7
:0CCA3C000000F03FA0DA00080000F0FF4E
:10CA480070B50C1C84B0051C0021201CFFF7F4F9FC
:10CA580000284ED1281CFFF7B7FC002803D02C1C57
:10CA6800201C04B070BD201CFFF7AEFC0028F7D1D5
:10CA78000021281CFFF7E0F90028F0D1281CFFF757
:10CA88009BFC00283DD1201CFFF796FC0028E6D12E
:10CA9800201CFFF78DFC011C061C281CFFF7A4FBBB
:10CAA80003A9FFF713FF0399301CFFF703FA011CD2
:10CAB800281CFFF7F9FA0021041C281CFFF774FB57
:10CAC800002820D0211C301CFFF76EF8002804D065
:10CAD800201C311CFFF7E8FA041C0021201CFFF77A
:10CAE800AFF80028BCD0201C311CFFF73FFA041C0B
:10CAF800B6E700F09DF8104B104C1B6801930360DB
:10CB0800AEE70E4CACE780231B06F118201CFFF79C
:10CB18004BF8002804D0201C311CFFF727FA041C0E
:10CB28000021201CFFF740FB002899D0201C311C55
:10CB3800FFF7BAFA041C93E7A0DA00080000C07FE8
:10CB4800F8B502000B000C00060049002148490D09
:10CB58000818132811DC00282EDB1F4901410C009E
:10CB68001C4014432FD08024240304410022E418DD
:10CB78008C43210014002000F8BD33280ADD8025ED
:10CB880014001900ED00A842F5D11000FFF770F865
:10CB98000400F0E7114DAC46012561446D42CD40DB
:10CBA800154210D03321081A323981408A1896422A
:10CBB80000D95C1CAA43DCE7DB0FDB07421C05D06D
:10CBC8001C000022D5E714001900D4E7044C002209
:10CBD8001C43CEE701FCFFFFFFFF0F00EDFBFFFF4B
:04CBE8000000F03F1A
:10CBEC00F8B5041E07DB0027002819DDFE208005A0
:10CBFC000D4D012606E044420127F7E76410043589
:10CC0C00002C05DD2642F9D02968FFF751F9F5E72C
:10CC1C00002F04D0011CFE208005FFF7E3FAF8BDBD
:0CCC2C00FE208005FBE7C04688DA000807
:10CC380000B5F6F791FA014B181800BD080000007E
:10CC4800F0B5DE4657464E464546E0B58FB08146BC
:10CC58000992002303604C1C0978002901D100F0D7
:10CC68006EFE060000F05BFE2200002780235B01B9
:10CC78009A46CB4C80239B009946F13BFF3B9C4650
:10CC88003033984606E05E2849D153461F4301E0F9
:10CC980043461F4315000132039228783028F2D802
:10CCA8001F2817D90300203BD9B2102912D88B00AE
:10CCB800E3589F4680231F43ECE780231B021F4352
:10CCC800E8E720231F43E5E763461F43E2E74B46B7
:10CCD8001F43DFE72A2822D1099B1A1D09921C68E5
:10CCE800002C34DBAB1C039A1078E243D2171440B3
:10CCF800002204922E282ED0742854D07A2852D09C
:10CD08006C2859D04C285DD0039368284ED11878E8
:10CD180068286AD00133039304231F4346E00024A4
:10CD28000300303B2100092B0FD88C0064186400E5
:10CD3800010030390919100001321300007804008D
:10CD4800303C092CF1D90C00CFE7039BCDE76442B6
:10CD580010231F43C6E718782A280DD1099A111DF8
:10CD680009911268049258780233049A002AC3DBA6
:10CD7800802252001743BFE701331A0001003039FF
:10CD88000929F5D804998B005B185B00010030393C
:10CD9800C91810000132130000780500303D092D34
:10CDA800F1D90491E1E75A1C0392187878280CD835
:10CDB80083007C4AD3589F465A1C03921878012353
:10CDC8001F43F3E7012217430393774B1D68002D98
:10CDD80001D100F09FFD09AB0193049B0093230050
:10CDE8003A003100A84700F095FD082217439A1C25
:10CDF80003925878DAE72521300002F0D5FC00F0DC
:10CE080089FD099B1A1D09921D78013C32002100F9
:10CE1800380001F050FE2900300002F0C5FCBA4687
:10CE28003AE03B0707D5099B1A1D09921B6832682F
:10CE38001A7000F06FFD099B1A1D09921B68326871
:10CE48001A6000F067FD099B1A1D09921B68994634
:10CE5800002B01D1554B9946554B3B409A46FB0553
:10CE680026D50499484602F0CDFC0500641B320023
:10CE78002100504601F01FFE6B1E9B46002D0BD073
:10CE88004F464D443978300002F08EFC0137BD42E0
:10CE9800F8D101235B429B465346DB0601D400F0E0
:10CEA80039FD32002100202002F09CFC00F032FD08
:10CEB800484601F00BFE0500D8E7099B1A1D0992A8
:10CEC8001B68802139404A425141494222229143FC
:10CED8008A4601329446E244DD321743F83A049216
:10CEE800002B01D100F0F3FC012280218901394097
:10CEF8008C460F218B460F2006A988464044A04641
:10CF0800654600F09AFC80239B011F4300239A4644
:10CF18003B060AD50300783B5A4253415B42202125
:10CF280019408A46234B9C46E244FB0501D5204B19
:10CF38001F407B0440D5099B1A1D09921B687A077C
:10CF480023D51BB2002B24DA5B422D2292463BE00C
:10CF5800802139404B42594149422F2399438A46FF
:10CF680001339C46E244FB05E3D5114B1F40E0E743
:10CF780000239A46FB05DCD50D4B1F40D9E78023DB
:10CF8800DB011F4300239A46D3E73A07DAD5FF228D
:10CF98001340BA062DD47A0616D52022924613E0FD
:10CFA800CCDA000810DB0008240E0020D4DE0008CC
:10CFB800FFFDFFFF58300000099B1A1D09921B68EE
:10CFC8007A0711D51B041B0CFA0501D400F0FBFBF2
:10CFD800CD4A17405838C2B2202A01D900F059FC6E
:10CFE8009000CA4A125897463A07EDD5FF221340D7
:10CFF800EAE72B229246E7E780239B011F43802321
:10D00800DB001F43099B0733072293431A000832AA
:10D01800099218685968FFF7DFF98046FB051AD5A9
:10D02800049B002B19D1C0252D013D40B84B9C46CF
:10D0380065446B426B4104930FE080239B011F43BF
:10D0480080231B011F43DDE780239B011F43C0236F
:10D058001B011F43D6E7062304934046FFF7ACF9AC
:10D06800002800D0CBE04046FFF7AEF90790002833
:10D0780000D0DEE04046FFF73BF9002800D0E1E0B1
:10D088004046051C0DA9FFF73BF90D9B5800C01839
:10D098000A2102F037FB0D900021281CFEF7CCFE78
:10D0A800002800D1D7E0C0231B013B401A00089399
:10D0B8008023DB009A420BD0C0231B019A4200D088
:10D0C800ABE10D9B049A934202DA043300DBA4E13E
:10D0D8000D9B5842FFF786FD011C281CFEF7EAFE4F
:10D0E800051C06900021FEF7A7FE002845D1281C44
:10D0F800FFF762F9002800D0C5E08649281CFEF732
:10D10800BFFE002816D00D9B01339946814B9A46E5
:10D11800A0464C4605945146281CFFF765F8051CA7
:10D1280001345146FEF7ACFE0028F3D1444606957B
:10D13800059B0D93069DFE218905281CFEF780FDA1
:10D1480000281AD00D9B013B9946724B9A46FE2344
:10D158009B0598464B46A1461C0005945146281C41
:10D16800FEF7A8FE051C013C4146FEF769FD0028B4
:10D17800F3D14C460695059B0D930499002907D0D9
:10D18800089B634A944663445A425341CB1A04931A
:10D19800049B5842FFF726FDFC218905FEF78AFE0D
:10D1A8000699FEF7E3FE051C5A49FEF769FE0028BA
:10D1B80000D082E00695049B002B00D195E08823DF
:10D1C8001B013B408022120193427FD0524B3B40CF
:10D1D8000593049B0533E41A013C01239A46FB049A
:10D1E80000D4D4E00D9D0321280002F0BDFA0231DD
:10D1F800042900D90FE18900484B5B589F4600215C
:10D208004046FEF71DFD002808D1BB040FD4444B4F
:10D218005A1C9146BA0605D5994603E0BB0404D4C6
:10D22800404B9946404B1F4016E6404BF9E7404BB0
:10D23800EEE7BB0404D43F4B99463B4B1F400BE63B
:10D248003D4BF9E760231F4380200006404418E760
:10D258000D9B01330D930D9B581CFFF7C3FC011C5C
:10D26800281CFEF7A1FF0028F2D102E00D9B013B2C
:10D278000D930D98FFF7B6FC011C281CFEF7E0FC87
:10D288000028F3D10FE70021281CFEF7D9FC00285D
:10D2980008D1BB040FD4224B5A1C9146BA0605D5B7
:10D2A800994603E0BB0404D41E4B99461E4B1F400D
:10D2B800D2E51E4BF9E71E4BEEE70D9B01330D93AC
:10D2C8001449281CFEF790FF069074E7049B092B6D
:10D2D80001DD092304930498FFF784FC0699FEF7FF
:10D2E800E9FDFEF7B9FD051E28D10B4B3B40059320
:10D2F800053C80231A003A4004923B4200D16CE777
:10D30800079B049368E7C046FFFDFFFFF4DC0008B5
:10D3180000F4FFFF00002041FFF7FFFF78DD000861
:10D32800BCDA0008ACDA0008FFFEFFFFA4DA000848
:10D33800B4DA0008C8DA0008C4DA00080A2101F0E3
:10D34800A5FB002900D041E7049B013B04930A2177
:10D35800280002F0F5F90500049B002BC5D00A212E
:10D3680001F094FB0029EFD030E701239A4609E049
:10D37800D0490698FEF79EFD0690013D0D95013CAB
:10D3880002239A46049AD343DB171A400492602377
:10D398003B405A1E9341E41A0D9802F02FFA632875
:10D3A80000DD013C069F381CFEF756FD0500FEF720
:10D3B800EBFE011C381CFEF777FE0690E343DB17F3
:10D3C80023409B4684239B00059A1A4200D1EAE039
:10D3D800059B9A0600D4F3E05B06DB17022119408F
:10D3E8002B31300002F0E0F9059BDB0600D4F0E0B9
:10D3F800B14B5344DB00B14A9F189146002401E128
:10D40800AF490698FEF756FD0690AB1E0D93023CF9
:10D4180003239A46B6E7DA46B4E77B0537D50D9B72
:10D428000E2B32DC0133049AD21A9146092A01DD07
:10D43800092291463A0602D54B46049327E0049AFE
:10D44800934271D09B4B9A46002398464B46A1467F
:10D458001C002000FFF7C6FB011C281CFEF72AFD54
:10D46800FC218905FEF782FDFEF778FF5146FFF79C
:10D47800E7FA4146FEF7E0FC002858D0013C002CB2
:10D48800E7D123004C46049301E0079B04938D4B9E
:10D498003B4005930D9B049A50421A00083A824279
:10D4A80049DD093B1800FFF79DFB01214942FEF7C2
:10D4B80039FF011C281CFEF759FD0690069B99466A
:10D4C8000D9B581CFFF78EFB011C4846FEF7D8FC45
:10D4D800002802D00D9B01330D930D98002847DBDF
:10D4E800092834DC4846FEF7B7FC0500FEF74CFE79
:10D4F800011C4846FEF7D8FD069000230D93002135
:10D50800092D4DD9704B01229246A8460122944616
:10D51800E24408331A00083A506888422DD8F5D1F9
:10D5280012684245F2D928E04B460493AFE723003E
:10D538004C460493ABE7FFF755FB01214942FEF740
:10D54800F1FE011C281CFEF711FD0690B6E703004A
:10D55800093B0D930923181AFFF744FB011C4846A1
:10D56800FEF7A8FCFEF778FC0500079B0693C6E7C4
:10D5780000230D93002501339A46049A130053445F
:10D588000D998C466344E41A80233B4013435A1E8A
:10D598009341E41A60233B405A1E9341E41A0DE775
:10D5A80001239A46E9E7002C00DC11E75C46013CC0
:10D5B8002021300002F0F8F8002CF8D1A34607E744
:10D5C800059B5B0600D40FE72021300002F0ECF841
:10D5D8000AE75B46002B00D10AE75C46013C302194
:10D5E800300002F0E1F8002CF8D1A34600E7AA4287
:10D5F8000ED93021300002F0D7F83B00083B4F45E8
:10D6080011D01F003A687B68002BF2D1A342EED0FC
:10D6180030210131C9B2AD1A002BEBD1A342F8D1A8
:10D62800AA42F6D9E6E780231B01059A14001C409C
:10D638001A424BD1049B002B55D1059B1B0600D5E4
:10D6480095E1059B5A0526D59904C9171F239943C7
:10D658006531300002F0A8F80D9B002B00DA9BE042
:10D668002B21300002F0A0F80D98632800DD9BE024
:10D678000A210D9802F046F801003031C9B2300095
:10D6880002F092F80A210D9802F06EF83031C9B212
:10D69800300002F089F85B46002B00D13AE15C4685
:10D6A800013C2021300002F07FF8002CF8D1A3467D
:10D6B80030E1C04600002041FFFFFF1FC0300008D6
:10D6C8000000C842FFFBFFFFD03000080D9B002B75
:10D6D800B0DD013B0D933021300002F065F80D9B61
:10D6E800002BF6DCA6E72E21300002F05DF8049B43
:10D6F8001D00092B00DD0925EB43DB171D40049BAA
:10D708005B1B9A46002C14D00D9BE81AFFF76AFAA7
:10D718000699FEF7CFFBFEF79FFB0400002D2ED0E5
:10D72800984BEB18DB00984A9846904400254746EA
:10D7380014E02800FFF756FA0699FEF7BBFBFEF740
:10D748008BFB0400EAE7A2420ED93021300002F038
:10D758002BF83B00083BB94511D01F003A687B689D
:10D76800002BF2D1AB42EED030210131C9B2A41A5C
:10D77800002BEBD1AB42F8D1A242F6D9E6E75346EB
:10D78800002B00D15DE75446013C3021300002F007
:10D798000BF8002CF8D154E72D21300002F004F8E2
:10D7A8000D9B5B420D935FE7642101F0ABFF010025
:10D7B8003031C9B2300001F0F7FF64210D9801F053
:10D7C800D3FF0D9154E701220492FFF703FC1900DF
:10D7D80001220F2006ADAC4660440725AC469946A9
:10D7E800002B58D065462B40303383541500C908A8
:10D7F8000B0001320029F5D1A9464CE09B460023D5
:10D8080099465B46002B0BD080231B023B402C25FE
:10D8180032005E46A0464C46B9461F00934627E0B4
:10D828000023994637E059461940584C615C8154A9
:10D8380011001B090132002B06D0002DF3D05946E8
:10D848001940534C615CF2E74446894623E00A21BB
:10D85800300001F01BF9303106AB10229B18195526
:10D8680001340A21300001F06BFF092E0CD90600A3
:10D87800002FECD003232340032BE8D106AB102262
:10D888009B181D550134E2E74F46A14644465E46C3
:10D8980001E000239946049B4A469D1AEB43DB1797
:10D8A8001D40641BA31A98465346FF2B12D9022326
:10D8B8005B429C46E0445346190AC9B2300001F065
:10D8C80073FF5346D9B2300001F06EFF04E0002325
:10D8D8009946E0E7002B50D132004146380001F06C
:10D8E800EAF832002900302001F07CFF4B46013B6A
:10D8F8009B460DD40AAC5D4665192978300001F0C5
:10D9080053FF2B00013DA342F7D101235B429B4605
:10D91800FB060DD4039B5C1C197800290ED0252921
:10D9280001D1FFF7A1F9300001F03EFF0394F1E7C0
:10D9380032004146202001F055FFEBE7B1464B4647
:10D948009B68002B07D04A461268494649688A42B4
:10D9580001D2002199544B4618680FB03CBC904640
:10D968009946A246AB46F0BD01204042F5E72E217C
:10D97800300001F019FF049DC1E601235B429C467B
:10D98800E0449EE7FFFFFF1FC030000874DA00087C
:04D9980064DA000845
:10D99C00000000000000000000000000000000007B
:10D9AC00000000000000000000000000000000006B
:10D9BC000100000002000000030000000400000051
:10D9CC00060000000700000008000000090000002D
:10D9DC00000000000000000000000000000000003B
:10D9EC000100000002000000030000000400000021
:10D9FC00004B0000000001000000000000000000CF
:10DA0C00000000000000000000000000000000000A
:10DA1C00000000000000000090D003000000000097
:10DA2C00000000000000000040420F00630069008D
:10DA3C00A086010004000A00B036C02BE02EC0F313
:10DA4C00C0DA0CFEF4014C1D581B54F248F44C1D6A
:08DA5C00581B54F248F40000CD
:10DA64003031323334353637383941424344454610
:10DA74003031323334353637383961626364656640
:04DA8400220000007C
:10DA8800000020410000C84200401C4620BCBE4C9B
:08DA9800CA1B0E5AAEC59D74B5
:04DAA0002100000061
:10DAA4002D494E46000000002D696E6600000000FE
:10DAB4002B494E46000000002B696E6600000000F2
:08DAC4004E414E006E616E0040
:10DACC0098CC0008DCCC0008DCCC0008BCCC0008EE
:10DADC00DCCC0008DCCC0008DCCC0008C2CC000894
:10DAEC00DCCC0008DCCC0008DCCC0008CACC00087C
:10DAFC00DCCC0008D0CC0008DCCC0008DCCC000866
:10DB0C00D6CC000870D90008D2CD0008D2CD0008C0
:10DB1C00D2CD0008D2CD0008D2CD0008D2CD00085D
:10DB2C00D2CD0008D2CD0008D2CD0008D2CD00084D
:10DB3C00D2CD0008D2CD0008D2CD0008D2CD00083D
:10DB4C00D2CD0008D2CD0008D2CD0008D2CD00082D
:10DB5C00D2CD0008D2CD0008D2CD0008D2CD00081D
:10DB6C00D2CD0008D2CD0008D2CD0008D2CD00080D
:10DB7C00D2CD0008D2CD0008D2CD0008D2CD0008FD
:10DB8C00D2CD0008D2CD0008D2CD0008D2CD0008ED
:10DB9C00D2CD0008D2CD0008FECD0008D2CD0008B1
:10DBAC00D2CD0008D2CD0008D2CD0008D2CD0008CD
:10DBBC00D2CD0008D2CD0008D2CD0008D2CD0008BD
:10DBCC00D2CD0008D2CD0008D2CD0008D2CD0008AD
:10DBDC00D2CD0008D2CD0008D2CD0008D2CD00089D
:10DBEC00D2CD0008D2CD0008D2CD0008D2CD00088D
:10DBFC00D2CD0008D2CD0008D2CD0008D2CD00087D
:10DC0C00D2CD0008D2CD0008D2CD0008D2CD00086C
:10DC1C00D2CD0008D2CD000800D0000842D00008B8
:10DC2C0050D00008D2CD0008D2CD0008D2CD0008CB
:10DC3C00D2CD0008D2CD0008D2CD0008D2CD00083C
:10DC4C00D2CD0008D2CD0008D2CD0008D2CD00082C
:10DC5C00D2CD0008D2CD0008D2CD0008D2CD00081C
:10DC6C00D2CD00080ECF0008D2CD0008D2CD0008CE
:10DC7C00D2CD0008D2CD0008D2CD0008D2CD0008FC
:10DC8C00D2CD0008D2CD0008D2CD0008D2CD0008EC
:10DC9C000ACE000886CF000806D0000848D000083D
:10DCAC0056D00008D2CD000886CF0008D2CD00088F
:10DCBC00D2CD0008D2CD0008D2CD00082ACE000863
:10DCCC0058CF0008C2CE0008D2CD0008D2CD000833
:10DCDC004ECE0008D2CD000878CF0008D2CD000877
:10DCEC00D2CD000814CF0008E8CE00089AD800085E
:10DCFC009AD800089AD800089AD800089AD8000830
:10DD0C009AD800089AD800089AD800089AD800081F
:10DD1C009AD800089AD8000804D800089AD80008A5
:10DD2C009AD800089AD800089AD8000804D8000895
:10DD3C009AD800089AD800089AD800089AD80008EF
:10DD4C009AD80008D6D70008E8CE00089AD8000860
:10DD5C009AD800089AD800089AD8000804D8000865
:10DD6C009AD800089AD80008E8CE000878D30008A2
:10DD7C0008D4000872D3000878D3000808D400082F
:10DD8C0011488546114C20680434004201D080476C
:10DD9C00F9E70F480F49091A082903DB0022026032
:10DDAC00043001600C480D49884205D002680430EB
:10DDBC0003B4904703BCF7E700208646EC460020EE
:10DDCC000021074A9047FEE70080002054FF00081E
:10DDDC00300E00203014002064DE000868DE0008DD
:04DDEC00D5850008D1
:10DDF0000448054988438546044880470448054946
:10DE00000160C3E70080002007000000958B000838
:08DE100008ED00E000300008FD
:10DE1800FEE7FEE7FEE7FEE7FEE7FEE7FEE7FEE7D2
:10DE2800FEE7FEE7FEE7FEE7FEE7FEE7FEE7FEE7C2
:10DE3800FEE7FEE7FEE7FEE7FEE7FEE7FEE7FEE7B2
:10DE4800FEE7FEE7FEE7FEE7FEE7FEE7FEE7FEE7A2
:0CDE5800FEE7FEE7FEE7FEE7FEE7FEE760
:04DE6400A58B000882
:10DE680084B0039002910020019002980C28009041
:10DE78001FD800987844007940008744061A1A1A77
:10DE88000B1A1A1A101A1A1A150003980068406B10
:10DE980001900FE003980068806B01900AE00398F6
:10DEA8000068C06B019005E003980068006C019061
:0ADEB80000E0FFE7019804B0704796
:10DEC20081B000900098806804210840800801B069
:02DED200704797
:07DED400286E756C6C29003B
:10DEDB00466972737420737461727420646574651F
:10DEEB00637465640A0070726576696F757320637D
:10DEFB006F6E6669672070726573656E740A004594
:10DF0B004550524F4D2046554C4C20524553544F83
:10DF1B005245210A00454550524F4D20464143542E
:10DF2B004F525920524553544F5245210A004545F3
:10DF3B0050524F4D2053544F524520434F4E46495C
:10DF4B0047210A0057726974696E6720534E210A84
:01DF5B0000C5
:10DF5C0083B00290019100920298406901990422C9
:10DF6C00114007228A409043009A8A40104302993C
:06DF7C00486103B070478C
:10DF820080B582B001900198806A0090009800F0FC
:06DF9200C8FD02B080BDD5
:10DF980080B582B001900198806A00900098816DE8
:10DFA8004022114381650098C16D04221143C16567
:0ADFB800009800F0AFFD02B080BD3C
:10DFC20081B000900098C068032189020840414254
:06DFD200484101B0704758
:10DFD80081B000900098806802210840400801B094
:02DFE800704780
:10DFEA0081B000900098006807218905084001B0B7
:02DFFA0070476E
:10DFFC0083B00290019100920298806A01991F22CD
:10E00C0011400F2213468B409843009B92061340FD
:0EE01C009A0E8A4010430299886203B0704742
:10E02A0010B584B0034603AC2070029101922078A7
:0EE03A0040B202990093F5F744FF04B010BD08
:10E0480080B586B00490039102920193684600213E
:10E058000170FFE704982421405C012804D1FFE700
:10E0680005A8022101706EE004982421012242547F
:10E07800FFE7FFE704982521405C01284FD1FFE71F
:10E08800049825210222425404980021C16304986F
:10E098000068016801229143016004980399029A7B
:10E0A800019BF6F745F80498006B002807D0FFE7B6
:10E0B8000498006801680E22114301600CE004987E
:10E0C80000680168042291430160049800680168AF
:10E0D8000A2211430160FFE70498406C0068C003FE
:10E0E800002808D5FFE70498406C01680122120255
:10E0F80011430160FFE70498006D002808D0FFE78E
:10E108000498006D01680122120211430160FFE7C3
:10E1180004980068016801221143016009E0FFE7E3
:10E128000498242100224254FFE768460221017026
:10E13800FFE7FFE70498242100224254FFE70098F4
:0EE1480005A90870FFE705A8007806B080BDA5
:10E1560010B583B013460C46029001A801806846AC
:10E1660002700078002805D0FFE701A80088029910
:10E17600886104E001A8008802998862FFE703B07D
:02E1860010BDCA
:10E1880083B00A46029001A80180029909690088B3
:10E19800014204D0FFE768460121017003E06846A8
:0EE1A80000210170FFE76846007803B0704761
:10E1B60082B00A4601906846018001994969008843
:10E1C600014205D0FFE7684600880199886204E0AD
:0EE1D6006846008801998861FFE702B0704733
:10E1E40083B0014602AA10700020019002986A468A
:10E1F4001070FFE7684600780A2808D3FFE7019803
:10E20400401C019000980A3869460870F2E70198AA
:0EE214000007000E69460978084303B0704702
:10E2220080B586B00490039102920498039B0299F0
:10E2320000910321C902002200F0B3FD002809D099
:10E24200FFE70498016E20221143016605A803210D
:10E2520001702CE00498039B029900918021002216
:10E2620000F01FFE002809D0FFE70498016E20226B
:10E272001143016605A80321017018E00498039B6D
:10E282000299009103214902002200F08AFD002830
:10E2920009D0FFE70498016E20221143016605A808
:10E2A2000321017003E005A800210170FFE705A822
:06E2B200007806B080BDFB
:10E2B80084B003900291019202981F210840012224
:10E2C800824000920098039A136A8343136201986C
:10E2D800029A0A40904003990A6A02430A6204B00B
:02E2E80070477D
:10E2EA0086B005900491039202930598016A102260
:10E2FA00914301620598806901900598006A00902F
:10E30A0001980321090288430190039800020199A8
:10E31A000143019101980F21090388430190029852
:10E32A00000380B20199014301910098A02188431A
:10E33A000090049800010840009901430091019857
:0EE34A000599886100980599086206B0704731
:10E3580086B005900491039202930598016A012200
:10E368001203914301620598C06901900598006AFB
:10E378000090019803210902884301900398000244
:10E3880001990143019101980F21090388430190E4
:10E398000298000380B20199014301910098052178
:10E3A80049038843009004980003084000990143FA
:10E3B800009101980599C86100980599086206B00E
:02E3C80070479C
:10E3CA0080B584B0039003986021405A01A908805F
:10E3DA00039884214058222834D1FFE70398006823
:10E3EA00406A694608800398806D029000980199F6
:10E3FA000840029908800398816D891C81650398F9
:10E40A005E21425A521E42520398405A002818D19D
:10E41A00FFE70398006801680922520191430160ED
:10E42A0003980068816801229143816003988421DE
:10E43A002022425003980021C166039800F083FF0E
:10E44A00FFE706E0039800688169082211438161A9
:06E45A00FFE704B080BDE5
:10E4600080B584B0039003986021405A02A90880C7
:10E47000039884214058222832D1FFE7039800688E
:10E48000406A01A908800198029908400399896DA2
:10E4900008700398816D491C816503985E21425A7A
:10E4A000521E42520398405A002818D1FFE70398A1
:10E4B00000680168092252019143016003980068D5
:10E4C0008168012291438160039884212022425077
:10E4D00003980021C166039800F03AFFFFE706E0C9
:10E4E000039800688169082211438161FFE704B045
:02E4F00080BDED
:10E4F20081B0009000982821405CC00700280CD011
:10E50200FFE70098006840680121490488430099A8
:10E51200CA6A104309684860FFE700982821405CF6
:10E52200800700280CD5FFE70098006840680121A9
:10E532000904884300990A6B104309684860FFE7A1
:10E5420000982821405C400700280CD5FFE700987E
:10E552000068406801218904884300994A6B10438E
:10E5620009684860FFE700982821405C00070028FE
:10E572000CD5FFE70098006840680121C903884371
:10E5820000998A6B104309684860FFE700982821C8
:10E59200405CC00600280CD5FFE700980068806840
:10E5A2000121090388430099CA6B104309688860F6
:10E5B200FFE700982821405C800600280CD5FFE781
:10E5C20000980068806801214903884300990A6C19
:10E5D200104309688860FFE700982821405C4006E4
:10E5E20000281DD5FFE70098006840680121090551
:10E5F2008843009A536C1843126850600098406C2C
:10E6020088420CD1FFE70098006840680321490561
:10E61200884300998A6C104309684860FFE7FFE766
:10E6220000982821405C000600280CD5FFE70098DE
:10E63200006840680121C90488430099CA6C1043EC
:0AE6420009684860FFE701B0704767
:10E64C0081B00090009880214058212823D1FFE709
:10E65C0000985621405A00280DD1FFE70098006819
:10E66C000168802291430160009800680168402293
:10E67C00114301600EE00098016D09780068816219
:10E68C000098016D491C016500985621425A521E92
:0AE69C004252FFE7FFE701B07047AC
:10E6A60083B00190FFE701987C21405C012804D1EA
:10E6B600FFE702A8022101702BE001987C210122CC
:10E6C6004254FFE7FFE70198802124224250019837
:10E6D60000680068009001980068026801239A4368
:10E6E600026000985A079043009001980022426603
:10E6F6000098019A12681060019820224250FFE7A4
:10E7060001987C2100224254FFE702A800210170F3
:0AE71600FFE702A8007803B0704787
:02E72000704740
:02E7220070473E
:02E7240070473C
:02E7260070473A
:10E7280084B003900398006902900398C068019030
:10E7380002980199884209D8FFE7039880680199EF
:10E74800401A02994018401E009005E0029801996D
:0EE75800C94308180090FFE7009804B070470E
:10E7660080B582B00190019800680168402291430B
:10E776000160019880212022425001980021016702
:0AE78600019800F0DEFD02B080BD36
:10E7900080B582B00190019826210C224254019844
:10E7A0000168FF22283282188B239B00C05A0090F8
:0EE7B00008461146009AF9F757F802B080BDEE
:10E7BE0081B0009000988B2189000022425001B058
:02E7CE00704792
:10E7D00081B0009000984521C90000224250009865
:06E7E000027501B0704754
:10E7E60084B00390029101920093029880300290C7
:10E7F60002980399009A88540098401C009001984A
:10E806000399009A88540098401C0090009804B020
:02E81600704749
:10E8180080B586B00590049105980499891EFCF787
:10E8280081FC02A908800598049A1018421E1278E3
:10E838001202801E0078101801AA1080088811881A
:10E84800884203D1FFE70498039003E00020C04307
:0AE858000390FFE7039806B080BDAF
:10E8620010B584B0039000200290039827300190E5
:10E872000398FFF7A3FF019800780399FF2228323B
:10E8820088540298401C0290039880180199029BB8
:10E892000C7800921A46234600F0F9FE0290039883
:10E8A20000994018029900F00EF80290029803991C
:10E8B2008B22920088500398FFF769FF0398FFF7B5
:06E8C20086FF04B010BD4A
:10E8C80080B586B00590049105980499FCF72AFC58
:10E8D80003A90880039802AA1070487801A9087053
:10E8E80002980599049A88540498401C0490019849
:10E8F8000599049A88540498401C0490049806B01A
:02E9080080BDD0
:10E90A0008D1004206D1F54204D801D3124201D1FE
:10E91A006D0D09D10020C143090DC904F0BDF9D11B
:10E92A001242F7D1640DF5D00020C14349054908C8
:10E93A00A6E000206146F0BDF0B50127FF070E00F2
:10E94A005E403E40B446BE0A4C18DD18F442D7D2A7
:10E95A00F542E4D2640DECD06D0DEAD06419C90217
:10E96A003943460DC0023143DB023B43DB0A10B494
:10E97A008E4685B297B26F43140C6C433E0CA419B1
:10E98A00260C2404BFB227439CB26C43A419190C69
:10E99A006943250CA4B249190D04090C6419000C29
:10E9AA0095B245433E0C76193743BFB2360C150C67
:10E9BA004543AD19A6B2240CAD192E0437432E0CCB
:10E9CA0036199DB24543AD19ACB22E0C89191D0CEE
:10E9DA0045436D182E04290C3443704680B295B213
:10E9EA0045433E0C76193743BFB2360C150C4543E6
:10E9FA00AD19A6B2AD19240C2E0437432E0C3619C4
:10EA0A009DB24543AD19ACB22E0C89191D0C454374
:10EA1A006D182E043443290C75462D0C90B26843A8
:10EA2A003E0C80190604BFB23E43070CA0B23F1841
:10EA3A00120C6A43D019020C80B2240CA4189AB2A0
:10EA4A006A43121914042043120C89181B0C6B43D5
:10EA5A00C91810BC01273D05294203D1B619404106
:10EA6A004941013CFF077D0D013D641B0BDB6D0035
:10EA7A00AC4209DA240500254208BE4168416141D9
:0AEA8A0066463143F0BD54E74EE745
:10EA94000A0010D00300400800E052008242FCD972
:10EAA400002000E05208934200D39B1A40418A425E
:0AEAB400F8D11900704700207047E8
:10EABE0010B5C30606D48005C017102318402030A9
:06EACE0000F08DFE10BDFA
:0EEAD400411C02780130002AFBD1401A704725
:10EAE2008446002A05D00B78037001300131013AC7
:06EAF200F9D160467047F7
:10EAF80081B00090009880680121084001B07047FB
:10EB080081B0009000988068012109070840000F33
:04EB180001B0704791
:08EB1C0081B0009001B07047C8
:08EB240081B0009001B07047C0
:10EB2C0080B584B0029002980068FFF74FFA00900D
:10EB3C0002980068FFF7DAFF002843D0FFE700983F
:10EB4C0000283FD1FFE70298006880680521084043
:10EB5C00012809D1FFE702980068F4F77DFE0298BE
:10EB6C000068032101600CE00298816D10221143B2
:10EB7C0081650298C16D01221143C16503A8027021
:10EB8C0024E0F4F761FB0190FFE7029800688068CD
:10EB9C00C007002815D0FFE7F4F756FB0199401A7F
:10EBAC0003280DD3FFE70298816D10221143816574
:10EBBC000298C16D01221143C16503A8027005E0E2
:10EBCC00E3E7FFE703A800210170FFE703A8007843
:04EBDC0004B080BD44
:10EBE00080B584B003900398806A02900298806D8B
:10EBF0005021084240D1FFE70298816D0122520264
:10EC00001143816502980068FFF7DBF900282FD0D7
:10EC1000FFE70298807E00282AD1FFE7029800686B
:10EC200000680007002822D5FFE702980068FFF778
:10EC300048F900280FD1FFE70298006841680C22CC
:10EC4000914341600298806D012108430902884385
:10EC5000029988650AE00298816D2022114381653E
:10EC60000298C16D01221143C165FFE7FFE7FFE78D
:10EC70000298F9F77FFA13E00298806DC006002829
:10EC800004D5FFE70298FFF749FF08E00298006DFE
:10EC9000406B03990190084601998847FFE7FFE719
:04ECA00004B080BD7F
:10ECA40082B001900091019800680721890588438A
:0CECB400009908430199086002B0704705
:10ECC00081B0009000988068C00F401E41424841CA
:04ECD00001B07047D8
:10ECD40081B00090009880680121084001B070471D
:10ECE40080B582B001900198F5F742F902B080BD79
:10ECF40080B582B0014601AA1070107840B200912C
:08ED0400F5F7D2F802B080BD62
:10ED0C0080B582B0014601AA1070107840B2009113
:08ED1C00F5F71AF902B080BD01
:0CED240081B001466A46108001B07047C3
:08ED300081B0009001B07047B2
:10ED380080B584B002900298002804D1FFE703A8A8
:10ED48000121017022E002983D21405C002808D191
:10ED5800FFE702983C2100224254029800F01AF87A
:10ED6800FFE702983D2102224254029804C801900C
:10ED78001046019A00911146F7F74CFC02980121C0
:10ED8800009A815403A800210170FFE703A80078C6
:04ED980004B080BD86
:08ED9C0081B0009001B0704746
:10EDA40010B586B0089C0490039102920193FFE78A
:10EDB400049800688068039908400299884267D0E3
:10EDC400FFE7039803214902884208D1FFE702982C
:10EDD400002804D1FFE704980068007BFFE701984E
:10EDE400401C002853D0FFE7F4F732FA0899401A80
:10EDF4000199884204D2FFE70198002846D1FFE731
:10EE0400049800684168E022914341600498406896
:10EE140041218900884215D1FFE7049880680121C7
:10EE2400C903884207D0FFE704988068012189025A
:10EE3400884207D1FFE704980068016840229143A3
:10EE44000160FFE70498806A0121490388420FD1D9
:10EE5400FFE7FFE704980068016801225203914329
:10EE6400016004980068016811430160FFE7FFE74F
:10EE740004985D2101224254FFE704985C2100229A
:10EE84004254FFE705A80321017005E0FFE78FE77F
:10EE940005A800210170FFE705A8007806B010BDA1
:10EEA400B0B586B00A9C15460490039102A802707E
:10EEB4000193FFE704980068806803990840401AAA
:10EEC4004142484102A90978884259D0FFE7019894
:10EED400401C002853D0FFE7F4F7BAF90A99401A06
:10EEE4000199884204D2FFE70198002846D1FFE740
:10EEF400049800684168E0229143416004984068A6
:10EF040041218900884215D1FFE7049880680121D6
:10EF1400C903884207D0FFE7049880680121890269
:10EF2400884207D1FFE704980068016840229143B2
:10EF34000160FFE70498806A0121490388420FD1E8
:10EF4400FFE7FFE704980068016801225203914338
:10EF5400016004980068016811430160FFE7FFE75E
:10EF640004985D2101224254FFE704985C210022A9
:10EF74004254FFE705A80321017005E0FFE799E784
:10EF840005A800210170FFE705A8007806B0B0BD10
:10EF940086B004900391029201A800210170FFE75A
:10EFA40004983C21405C012804D1FFE705A8022114
:10EFB400017033E004983C2101224254FFE7FFE74B
:10EFC40002980028009004D0FFE7009804280BD092
:10EFD40016E004980068806E0F2188430399084363
:10EFE4000499096888660FE004980068806E0F2110
:10EFF400090288430399084304990968886603E071
:10F0040001A801210170FFE7FFE704983C210022D9
:10F014004254FFE7019805A90870FFE705A80078A6
:04F0240006B070477B
:08F0280081B0009001B07047B7
:08F0300081B0009001B07047AF
:10F0380080B588B0069005910492FFE706983C21B8
:10F04800405C012804D1FFE707A80221017091E084
:10F0580006983C2101224254FFE7FFE706983D212C
:10F0680002224254049800281AD1FFE70698006843
:10F0780005990A684B68C968039111461A46039BAB
:10F08800F7F748FB0698006881690C229143816173
:10F0980005988068069909688A6902438A615BE075
:10F0A800049804281CD1FFE70698006805990A68A7
:10F0B8004B68C968029111461A46029BFFF711F97D
:10F0C800069800688169032292029143816105983C
:10F0D80080680002069909688A6902438A613AE0F1
:10F0E800049808281AD1FFE70698006805990A6865
:10F0F8004B68C968019111461A46019B00F03EF819
:10F1080006980068C1690C229143C161059880681E
:10F1180006990968CA690243CA611BE00698006833
:10F1280005990A684B68C968009111461A46009B00
:10F13800FFF70EF906980068C1690322920291430D
:10F14800C16105988068000206990968CA69024386
:10F15800CA61FFE7FFE7FFE706983D210122425415
:10F16800FFE706983C2100224254FFE707A8002148
:0CF178000170FFE707A8007808B080BD18
:10F1840086B005900491039202930598016A0122C6
:10F194001202914301620598C06901900598006AC2
:10F1A4000090019803218843019003980199014339
:10F1B40001910198F0218843019002980001C0B2A6
:10F1C4000199014301910098052149028843009067
:10F1D40004980002084000990143009101980599A0
:0CF1E400C86100980599086206B07047E9
:08F1F00081B0009001B07047EE
:08F1F80081B0009001B07047E6
:10F20000B0B586B00A9C15460490039102A802701E
:10F210000193FFE704980068C06903990840401A09
:10F220004142484102A90978884231D1FFE70A9852
:10F23000401C00282BD0FFE7F4F70CF80199401A86
:10F240000A99884204D8FFE70A9800281ED1FFE7F0
:10F250000498006801680D225201914301600498EE
:10F2600000688168012291438160049880212022F6
:10F270004250049884214250FFE704987C210022E8
:10F280004254FFE705A80321017005E0FFE7C1E74D
:10F2900005A800210170FFE705A8007806B0B0BD01
:08F2A00081B0009001B070473D
:08F2A80081B0009001B0704735
:10F2B00082B0019001988021405821283ED1FFE77B
:10F2C00001986A21405A69460880FFE7684600882D
:10F2D000002832D0FFE701985621405A00280ED16D
:10F2E000FFE70198006881680122D205914381609F
:10F2F0000198006801684022114301601DE00198F7
:10F300000068C069000600280FD5FFE70198016D6D
:10F310000978006881620198016D491C01650198B6
:10F320005621425A521E425200E0FFE7FFE7FFE734
:10F330000098401E69460880C8E7FFE702B07047A2
:08F3400081B0009001B070479C
:08F3480081B0009001B0704794
:08F3500081B0009001B070478C
:10F3580080B582B0014601AA1080108801225202AD
:10F36800904203D1FFE700F02FF8FFE702B080BD1D
:0CF3780080B501204002F5F7CBFA80BD03
:08F3840080B5F3F7EFFE80BD38
:04F38C00FFE7FEE7B2
:10F3900081B0009000982121C900415881670098F0
:10F3A000CE21415A7C2281520098CC21415A7E22A2
:10F3B00081520098D42141588022815001B0704779
:10F3C00080B50520000708210122FEF7C4FE80BD9C
:08F3D00080B5FAF783F880BD57
:10F3D80080B588B00790069105920798C068039099
:10F3E800079880680399401A029002980599884204
:10F3F8000ED9FFE707984068039940180699059ABF
:10F40800FFF76BFB0399059A8918079AD1601DE0ED
:10F418000298049007984068039940180699049A3E
:10F42800FFF75BFB0599029A891A049107994968C5
:10F43800069A029BD218049B0190084611461A4668
:10F44800FFF74BFB0499079AD160FFE708B080BD2E
:10F4580080B58AB009900891079200200590099814
:10F46800C0680390FFE7099800690490049803991D
:10F47800884206D9FFE704980399C94308180690FB
:10F4880008E0099880680399049A891AC9430818FA
:10F498000690FFE7069809998968039A891A8842AD
:10F4A80003D2FFE70698029005E00998806803995F
:10F4B800401A0290FFE7029806900698079988423A
:10F4C80003D2FFE70698019002E007980190FFE752
:10F4D8000198069009984068039940180899069A77
:10F4E800FFF7FBFA0699059A511805910699089AAB
:10F4F800511808910699079A511A07910699039A83
:10F50800511803910399099A9268914203D1FFE730
:10F5180000200390FFE703980999C860FFE7079860
:0CF528000028A0D1FFE705980AB080BDC4
:10F5340083B080B5A3B0279326922591229025A865
:10F544000090229A009B01A8802100F071F921907B
:10F554002198812806DBFFE7002001A98022FBF720
:10F5640035FA0AE02198012806DBFFE7219A0020FA
:10F5740001A9FBF72BFAFFE7FFE7219823B080BC32
:08F5840002BC03B08E46704783
:10F58C0081B00090009880214058212823D1FFE7BA
:10F59C0000985621405A00280DD1FFE700980068CA
:10F5AC000168802291430160009800680168402244
:10F5BC00114301600EE00098016D097800688162CA
:10F5CC000098016D491C016500985621425A521E43
:10F5DC004252FFE70CE000980068016880229143DA
:10F5EC000160009800680168402211430160FFE748
:04F5FC0001B07047A3
:10F6000081B000900098007D0121084001B0704752
:10F61000B0B588B00790069105920493059800282C
:10F6200004D0FFE70598012803D1FFE701200290ED
:10F6300002E002200290FFE702980930039005984B
:10F64000002804D0FFE70598012804D1FFE70398BC
:10F65000401C0390FFE707980499069A059B029CBB
:10F66000039D01950094FBF78DFB079800214177DE
:10F670000798818407980184079826228154079867
:10F6800001770798C18307982222815408B0B0BD42
:10F6900010B588B01C4607900691059204A8037027
:10F6A00006984078039003980328019008D0FFE75C
:10F6B000019806280DD0FFE70198102812D01AE013
:10F6C00007980699059A04AB1B78FBF707FC029094
:10F6D00019E007980699059A04AB1B78FBF7C2FC62
:10F6E000029010E007980699059A04AB1B78FBF787
:10F6F0005FFD029007E007980399059B0122FFF741
:0CF7000072F80290FFE7029808B010BDFC
:10F70C00CA1751408B1A17D0C1174A4004B448404D
:10F71C00411A48081A0000E052008242FCD900202D
:10F72C0000E05208914200D3891A40419A42F8D124
:0CF73C0004BC5040801A70470020704749
:10F748000A000FD00300400800E052008242FCD9B2
:10F75800002000E05208934200D39B1A40418A429D
:08F76800F8D170470020704742
:10F77000CA1751408B1A19D0C11706B44840411A14
:10F7800048081A0000E052008242FCD9002000E044
:10F790005208914200D3891A40419A42F8D10CBCD8
:10F7A00053405840C01A5140891A70470020704792
:10F7B00070B504000800A568002D0AD022686168B1
:10F7C000531C5B1A5E1EB3415B4218408A4209D249
:10F7D000A854E368002B05D0226861688A4201D2F0
:0CF7E0002100984723680133236070BDAE
:10F7EC0070B516004C1E06D4C5B229003000FFF7C8
:08F7FC00D9FF013CF9D270BDF8
:08F80400C317C01858407047FB
:10F80C000378002B0CD000290CD0411803000133D5
:10F81C001A78002A02D08B42F9D10B00181A7047C3
:08F82C000300FBE70300F9E70C
:10F8340010B584B00C0011001A0002900023039349
:0CF8440001946846FDF7FEF904B010BD09
:10F8500000228446002903D0027001300139FBD117
:04F860006046704747
:10F8640002000B78013113700132002BF9D170477B
:10F874004953454E534F525F3530303A20496E69F3
:10F88400740A0066756C6C20726573746F72652EF1
:10F894002E2E0A007265616420636F6E6669672E9E
:10F8A4002E2E0A00666163746F7279207265737418
:10F8B4006F72652E2E2E0A004144533132363020A9
:10F8C400496E69740A00554E4B4E4F574E20434FB4
:10F8D4004D4D414E440A00537461727420656E614B
:10F8E400626C6520726561646F75742070726F74E8
:10F8F400656374696F6E0A00466C61736820756E87
:10F904006C6F636B206572726F720A00466C617370
:10F9140068206F6220756E6C6F636B206572726F06
:10F92400720A002E2E2E466C61736820756E6C6F01
:10F93400636B0A002E2E2E456E61626C65206C6F1F
:10F94400636B206572726F720A00466C6173682083
:10F954004F7074696F6E62797465206C6F636B6548
:10F96400640A00466C61736820206C6F636B656485
:10F974000A002E2E2E456E61626C65206C6F636BDF
:10F984002070726F636573732066696E697368654E
:10F99400640A002E2E2E466C617368206C6F636BB4
:10F9A40020616C7265616479206163746976650AAB
:10F9B400002E2E2E466C61736820756E6C6F636B1F
:10F9C40065640A002E2E2E466C617368206F6220D7
:10F9D400756E6C6F636B65640A00466C61736820B6
:10F9E4004F7074696F6E627974652070726F67729C
:10F9F400616D6D206661696C65640A00466C6173B3
:10FA040068204F7074696F6E627974652070726FCC
:10FA14006772616D6D65640A002E2E2E44697361F0
:10FA2400626C65206C6F636B2070726F63657373B7
:10FA34002066696E69736865640A0050524F5445C4
:10FA44004354494F4E3A204F425F5244505F4C4515
:10FA540056454C5F300A0050524F54454354494F69
:10FA64004E3A204F425F5244505F4C4556454C5FDE
:10FA7400310A0050524F54454354494F4E3A204F97
:0FFA8400425F5244505F4C4556454C5F320A007A
:10FA93004F5554505554535F4C56505F4241545444
:10FAA3004552595F554E444552564F4C5441474574
:10FAB3000A004F5554505554535F4C56505F4F56A0
:10FAC300455243555252454E540A004F55545055D2
:10FAD30054535F4C56505F5348554E545F4F5645F1
:10FAE3005254454D50455241545552450A004F55C5
:10FAF30054505554535F4C56505F434849505F4FE1
:10FB030056455254454D50455241545552450A00AD
:10FB13004F5554505554535F4C56505F5348554EB0
:10FB2300545F554E44455254454D504552415455EA
:10FB330052450A004F5554505554204C5650204FAF
:10FB43004B0A004F5554505554535F4F56505F4224
:10FB53004154544552595F4F564552564F4C5441A8
:10FB630047450A004F5554505554535F4F56505F05
:10FB73004F56455243555252454E540A004F555421
:10FB8300505554535F4F56505F5348554E545F4F33
:10FB930056455254454D50455241545552450A001D
:10FBA3004F5554505554535F4F56505F4348495037
:10FBB3005F4F56455254454D504552415455524559
:10FBC3000A004F5554505554535F4F56505F534896
:10FBD300554E545F554E44455254454D5045524140
:10FBE300545552450A004F5554505554535F4F5680
:10FBF300505F434849505F554E444554454D504529
:10FC03005241545552450A004F5554505554204FB4
:07FC13005650204F4B0A0080
:10FC1A004552524F52205452494D4D494E47205653
:07FC2A00414C5545530A004F
:0AFC310012000000000000000000B7
:10FC3B004552524F52204144535F313236305F535D
:10FC4B00657444617461526174650A004552524F88
:10FC5B0052204144535F313236305F5365744469EF
:10FC6B00676974616C46696C7465720A002D2D2D81
:10FC7B00204761696E202043414C202D2D2D0041E2
:10FC8B0044535F313236305F42617474657279432D
:10FC9B00757272656E744761696E43616C696272ED
:10FCAB006174696F6E53746172743A204552524F8E
:10FCBB005220494E2043414C4942524154494F4EE8
:10FCCB002C204E4F205245464552454E434520432E
:10FCDB00555252454E54210A0049202877697468C1
:10FCEB006F757420636F6D70656E736174696F6E81
:10FCFB00293D25660A0049205265666572656E7A54
:10FD0B003D25660A00547368756E743D25660A00BE
:10FD1B0054736869703D25660A004B6F7272656B90
:10FD2B0074757266616B746F723D25660A002D2DBA
:10FD3B002D204761696E202043414C20454E4445A0
:10FD4B002D2D2D002D2D2D204761696E20447269BC
:10FD5B0066742043414C202D2D2D00416374756139
:10FD6B006C20543D256620B0430A0064656C7461B9
:10FD7B0020543D256620B0430A0041637574616CC5
:10FD8B0020493D2566204128776974686F7574207A
:10FD9B006761696E2074656D70206472696674208A
:10FDAB00636F7272656374696F6E290A00526566C0
:10FDBB0020493D25660A004B6F7272656B74757234
:10FDCB0066616B746F723D2566205B2031202F209E
:10FDDB0043656C736975735D0A002D2D2D2047618A
:10FDEB00696E2044726966742043414C20454E4431
:10FDFB0045202D2D2D004610004552524F522041CB
:10FE0B0044535F313236305F536574496E7465729B
:10FE1B006E616C5265666572656E63650A0045526C
:10FE2B00524F52204144535F313236305F53657429
:10FE3B00436F6E76657273696F6E4D6F64650A0002
:10FE4B004552524F52204144535F313236305F534B
:10FE5B00657443686F704D6F64650A004552524F6D
:10FE6B0052204144535F313236305F496E707574A6
:10FE7B004D757853656C6563740A00693D25662082
:10FE8B00412E206973743D25662C2066733D2566D3
:0AFE9B002C206454733D25660A0014
:0AFEA500470000000000000000000C
:0EFEAF0075617274206572726F72200A0D0008
:10FEBD0063616C696C62726174696F6E2076616CDE
:10FECD007565203A202564003A2020206672657100
:10FEDD0075656E6379203A2025640A0056616C754C
:10FEED0065206E6F742076616C69640A00467265D8
:10FEFD007175656E6379204D6561737572656420EA
:10FF0D003D2025640A006869676865737420667210
:10FF1D00657175656E63792025640A006C6F776570
:10FF2D00737420206672657175656E637920256422
:02FF3D000A00B8
:10FF3F005465726D696E616C00525454005345479D
:04FF4F0047455200D0
:10FF54000900010800000020040000000900010855
:10FF64008C000020A00D00001F00010804000020E8
:0CFF740080FF0008880000000000000072
:10FF800088B00590049103A80021017005980290A3
:10FF900004980190174801680122920411430160FE
:10FFA000EFF3108006900698009072B6FFE703A862
:10FFB00000783F280FD8FFE7019800680299086091
:10FFC0000198001D01900298001D02900398401CAA
:10FFD00003A90870EBE7FFE707480068C0030028A3
:10FFE00001D5FFE7F8E700980790079880F310889D
:10FFF00008B07047142002401020024001000000A9
:020000040801F1
:08000000040000000024F400DC
:10000800206861680834094204D000220270013077
:060018000139FBD1704725
:10001E0020686168A2680C34124205D00B78037018
:0A002E0001300131013AF9D17047A9
:040000050800DDF121
:00000001FF
